:020000040800F2
:2000000080150020D9000008111300083312000800000000000000000000000000000000D1
:20002000000000000000000000000000251300080000000000000000131300082713000810
:20004000EB000008EB000008EB000008EB000008EB000008EB000008EB0000083D070008AF
:2000600000000000EB000008EB00000800000000EB000008EB000008EB00000800000000C1
:20008000EB000008EB00000800000000EB00000800000000EB000008EB000008EB000008AE
:2000A00000000000EB000008EB000008EB0000085D170008EB000008EB0000080000000005
:2000C0000448854600F050F800480047C9190008C046C046801500200448804704480047F1
:2000E000FEE7FEE7FEE7FEE7FEE7FEE745130008C100000830B50B46014600202022012475
:2001000009E00D46D5409D4205D31D469540491B2546954040191546521E002DF1DC30BDF0
:2001200003460B439B0703D009E008C9121F08C0042AFAD203E00B780370401C491C521EFC
:20014000F9D27047D2B201E00270401C491EFBD270470022F6E710B513460A4604461946E9
:20016000FFF7F0FF204610BD064C0125064E05E0E36807CC2B430C3C98471034B442F7D3FF
:20018000FFF7A2FFB81A0008D81A0008FEB504460D4600270026281B800A0190281B800531
:2001A000800D009000BF15E0124A012080022118204600F0EFFC012109030E4800F01CF86D
:2001C0008619012109030B48FFF7C3FF0120800224187F1C01988742E6D300982118054A92
:2001E000204600F0D7FC0348009900F005F886193046FEBD2802002010B502460B4600216C
:20020000002000BF02E0545C2018491C9942FAD310BD0000FEB50446002500270020029060
:200220000190009000268A20005B0C2807D08821085B01230022114600F0DAFBFEBD00BF7F
:20024000E81C205C0006A91C615C09040843691C615C09020843615D084307462D1D3A4884
:2002600000F0A6FC02900298C007C00F029002983840002804D101210198084301904CE0C6
:20028000E81C205C0006A91C615C09040843691C615C09020843615D08432C4988612D1DB5
:2002A000084680691121C902884204D9022101980843019031E0002611E00120B04038401A
:2002C00000280BD0B0002249085820494860B0001F4908581D4988600E7002E0761C002EA9
:2002E000EBD000BF1949886800F0FEFB002804D004210198084301900FE0E81C205C00063E
:20030000A91C615C09040843691C615C09020843615D08430D49C86000BF00BF01980028A5
:2003200002D19420019005E01C210848FFF711FF012000908821085B042201A9009B00F015
:2003400057FB00BF7AE7000000AF0008CC0000200800002038B50446002000900025012132
:200360000098084300908821085B2B460422694600F03EFB38BD0000F8B5044600200090F3
:2003800003250026084800F013FC054600950098C007C00F00908821085B334604226946C8
:2003A00000F026FBF8BD000000AF0008F0B585B004460025002004900390029001900026E7
:2003C00000908A20005B082808DA8821085B01230022114600F00CFB05B0F0BD00BFE81CB1
:2003E000205C0006A91C615C09040843691C615C09020843615D084304900498FB2801D1DB
:20040000049804902D1D594841690498814204D0012103980843039091E054484069401C37
:2004200052494861E81C205C0006A91C615C09040843691C615C09020843615D08430290E5
:200440002D1D8A20005B461B48480069801947490861084600698969884204D91021039845
:20046000084303906BE0B007800F002804D0202103980843039062E0611932463C48FFF7A9
:200480004FFE802E08D2B7B204E0FF203849C855781C87B2802FF8DBB1030A0C33498868F8
:2004A000334900F055FB002806D002200390022103980843039042E02C4A926891192B4A80
:2004C00090682C4A00F066FB31462A48FFF794FE019002990198884202D0082003902EE0C2
:2004E0002248806880192149886008460069896988421AD11D4A52681C4B9B69D1181B4A87
:200500005068FFF743FE01901848C1680198814208D18020039018480068012108431649D6
:20052000086001E04020039009E01049886800F0DBFA002802D0FF200130009000BF00BF30
:200540000398002808D00398802805D0012000901C210648FFF7FDFD8821085B042203A9DE
:20056000009B00F045FA00BF36E70000CC000020A80100202801002004000020F8B50446BC
:20058000002500200090002600F0C2FC054600958821085B33460422694600F029FAF8BDB0
:2005A000F0B502460B460021002400250C2B01DA481EF0BD505CFD280BD1481C105CFC28CD
:2005C00007D1881C105CFB2803D1C81C105CFA2802D00020C043ECE7081DC1B2181FC3B2BE
:2005E000481C105C0002565C30430546881CC1B2981EC3B2481C105C0002565C30431C4E16
:200600003081881CC1B2981EC3B2A81E86B2184846814089882811DC0BE008464E1CF1B216
:20062000165C2046671CFCB2114F803F3E54581EC3B20F484089A042EFDC02E00020C04343
:20064000B7E7042B0EDB505C04280BD1481C105C032807D1881C105C022803D1C81C105CFF
:20066000012802D00020C043A3E70020A1E70000C000002010B514480068002800D110BDFB
:20068000114801781148FFF78BFF002803D000200D490860F3E70E4800F024F80D480088BD
:2006A00081B20D4801F0CAF90020074908600B480078C007C00F002804D0094908780121D5
:2006C00000F0BAFD00BFDAE71000002028120020400000200C000020E800002004000020B1
:2006E000CC00002010B504468820005B7038030001F05AF80604080C101814182046FFF740
:2007000029FE17E02046FFF737FE13E02046FFF781FD0FE02046FFF749FE0BE02046FFF784
:200720002DFF07E08821085B01230022114600F05FF900BF00BF002010BD00004020084999
:20074000C9680140814201D1012100E00021002904D040200249C86000BF00BF704700006A
:200760000018024000B500200649486000F0D6FA0548406904210843034948610348C10626
:20078000086000BD64130020002002402143341200B5034600200D49486000F0BFFA0C4878
:2007A0004069022108430A494861FF20186000BF07480069012109040840002805D0044858
:2007C0000069C007C00F0028F2D000BD6413002000200240F0B589B004460F460020089045
:2007E00000250790069002900390049005900190A007800F002802D0681E09B0F0BD18484C
:20080000844203D80120C006844202D20020C043F3E70120C006201A07900798C009089001
:200820000898C0010121C90645182E460220029003950120059001A902A800F0BDF9002871
:2008400002D00020C043D8E73A462946012000F02BFA002802D00020C043CEE70020CCE71A
:2008600000C00008F0B5A9B004460F4600202890279026900025259021902290239024902A
:2008800000260090A007800F002802D0681E29B0F0BD1F48844203D80120C006844202D2DD
:2008A0000020C043F3E70120C006201A28902898C00926902698C0010121C9064518601BDB
:2008C00027900095002604E00098805D01A98855761C802EF8D3022021902295012024905C
:2008E00025A921A800F068F9002802D00020C043CDE701A927980F5001AA2946012000F04C
:20090000D3F9002802D00020C043C0E70020BEE700C00008F0B502460B46002014461D469F
:20092000144E766901273E43124F7E6100BFEFF31086314672B60EE02E6826602D1D241D22
:20094000461CF0B21F2806D10A4E76690127FF043E43084F7E612028EED300BF054E3669A2
:2009600001273F043E40002EF8D100BF81F3108800BFF0BD0020024000B5034600F0CEF949
:200980000B4840690121C902084309494861FF20186000BF0648006901210904084000287C
:2009A00005D003480069C007C00F0028F2D000BD0020024070B5044600F0A4FA051905E00F
:2009C00000F0A0FAA84201D3032070BD06480069012109040840000C0028F1D103480249C5
:2009E00008610020F1E700000020024011800000FFB5002004240023FD260746401C384D33
:200A0000EE55FC260746401CEE55FB260746401CEE55FA260746401CEE55002901D0A518B5
:200A2000ACB20546471CB8B22D4F7C55FF252D0225402E120546471CB8B2294F7E55FF2673
:200A40000136009D3543EEB20546471CB8B2244F7E55FF260136009D3543FF263602354009
:200A60002E120546471CB8B21D4F7E55039DEEB20546471CB8B21A4F7E55FF263602039D4E
:200A800035402E120546471CB8B2154F7E55002908D0002304E0CD5CC618114FBD555B1C5A
:200AA0009342F8D38518A8B204260546471CB8B20B4F7E5503260546471CB8B2084F7E55C5
:200AC00002260546471CB8B2054F7E5501260546471CB8B2024F7E55024D2860FFBD0000B9
:200AE000E80000200C00002010B586B00446002001906006400E002803D00020C04306B044
:200B000010BD0220029003940120059001A902A800F052F8002803D002A0019900F034FE20
:200B20000020ECE748414C5F464C41534845785F4572617365204572726F722C5061676541
:200B40004572726F72203D2025640D0A00000000F8B504460E4615460027A80000190C498B
:200B6000884201D9781EF8BDA007800F002802D00020C043F7E731462046FFF72BFE002831
:200B800001D1241D02E00020C043ECE70020EAE700C0000870B505460E462B4605E0184639
:200BA00000F006F8044610C21B1DB342F7D370BD0146086870470000F8B504460E46012726
:200BC000002500BF36480078012801D10220F8BD01203349087000BF2068012815D17D2061
:200BE000C000FFF7E7FE002852D1FFF7BBFD7D20C000FFF7DFFE074600F090F82948406952
:200C0000042188432749486142E02068022825D17D20C000FFF7CEFE002839D1401E3060C2
:200C2000656814E02846FFF7B3FD7D20C000FFF7C1FE074600F072F81A484069022188432D
:200C400018494861002F01D0356006E08035E068C00161684018A842E4D819E020680328DE
:200C600016D17D20C000FFF7A5FE002810D1A068FFF782FE7D20C000FFF79CFE074600F0E6
:200C80004DF8084840690121C90288430549486100BF00200249087000BF384697E700000A
:200CA0006413002000200240F8B507460D461646012400BF17480078012801D10220F8BD05
:200CC00001201449087000BF7D20C000FFF772FE0446002C16D100F021F831462846FFF75B
:200CE00019FE7D20C000FFF765FE044600F016F8094840694008400007494861002C01D067
:200D00002046DCE700BF00200249087000BF2046D5E70000641300200020024000200949BC
:200D20004969C90FC90700290BD00749054A91600649916011464969C90FC907002900D0DB
:200D4000012070470020024023016745AB89EFCD70B503460022CBE0012696400C68344079
:200D6000002C71D04D68022D02D04D68122D15D1D508AE001D462035A8595507EE0E0F25A6
:200D8000B5400646AE4330465607F60E0D69B5402843D508AD001E46203670511868560099
:200DA0000325B5400646AE4330460D79AD07AD0F5600B540284318604D68012D08D04D68CF
:200DC000022D05D04D68112D02D04D68122D18D1986856000325B5400646AE4330465600F1
:200DE000CD68B540284398605868012595400646AE43304610264D6835402D099540284322
:200E00005860D86856000325B5400646AE43304656008D68B5402843D860012636074D68B8
:200E20003540B54263D1354D9608B600A8599507EE0E0F25B5400646AE43304605252D0769
:200E4000AB4202D1002506E051E02D4DAB4201D1012500E002259607F60EB5402843274DBB
:200E60009608B600A851254D203528680546A5432846012636044D683540B54202D105468D
:200E8000254328461D4D2035286068680546A5432846012676044D683540B54202D10546E4
:200EA00025432846154D20356860144D603D28680546A5432846012636054D683540B5422B
:200EC00002D10546254328460C4D603D286068680546A5432846012676054D683540B5426C
:200EE00002D1054625432846044D603D6860521C0D68D540002D00D02EE770BD6018024057
:200F00000004005001480068704700002C0000200148006870470000000EFF1F0348006882
:200F20000349096840180149086070472C0000203400002010B50024032000F009F800286E
:200F400001D0012401E000F033F8204610BD0000F8B5044600251348006800281ED011481E
:200F600001687D20C000FFF7C5F8074639460E480068FFF7BFF8064600F052F800280BD137
:200F8000042C07D200222146401E00F025F80748046004E0012502E0012500E0012528461B
:200FA000F8BD0000340000202800002030000020704700000146002909DB00BF00BFCB0636
:200FC000DB0E01229A40034B1A6000BF00BF00BF7047000000E100E070B504460D46164690
:200FE0002946204600F0EEFB70BD000001480068704700002800002000B5FFF7F7FF064976
:201000008968072212031140090B8900034A515CC906C90EC84000BD00100240981A000842
:2010200070B504462546681E0949884201D901200CE0681E074948610321081F00F0C2FBD6
:2010400000200449886107200861002070BD0000FFFFFF0000E000E00146044A1068044A45
:201060000A600022014B1A6070470000380000207C13002010B509490968202211402029FC
:201080000AD101684968CAB205490B680968491C034C21600349CA5410BD000000440040BD
:2010A000380000207C13002010B50446002C01D1012010BDA069002800D000E000BF4D2021
:2010C000005D002805D100214C200155204600F030F824214D2001552068C068012149032E
:2010E00088432168C860204600F02EFA206A002802D0204600F03CF9206800690121C90209
:201100008843216808612068406908218843216848612068C0680121490308432168C860A1
:201120000020206520214D2001554E2001550020BFE77047FFB583B004460D4617460020C4
:2011400001904D20005D202871D1002D01D0002F02D1012007B0F0BD01210903A068884225
:2011600008D12069002805D1E807C00F002801D00120EFE700BF4C20005D012801D10220BC
:20118000E8E701214C20015500BF0020206521214D200155FFF7B6FE01902786678601213C
:2011A0000903A068884205D12069002802D10026029502E02E46002002901EE00698009006
:2011C000002280212046019B00F090FA002801D00320BFE7002E09D102980088C005C00D52
:2011E000216848600298801C029003E0307821684860761C608E401E6086608E0028DDD1B2
:2012000006980090002240212046019B00F06EFA002801D003209DE720214D20015500BF60
:2012200000214C20015500BF002093E7FFE7022090E700BFFEE70000F8B506460D462D4C8A
:20124000012D19D100272C48FFF74EFC002801D000BFFEE701212848FFF704FB002801D07E
:2012600000BFFEE72448FFF7A3FC0746781C002801D100BFFEE700BF20484068000C00046B
:201280000121C90340181E49096908431B49486000BF1A4800680121890208408842F8D1C7
:2012A00018480068C0688910884316490968C8601448006840694008400012490968486178
:2012C00010480068C068202188430E490968C86020680D49084001214907884209D1206866
:2012E00080F3088800BF606808490860084600688047F8BD0020000800AF00080010024048
:20130000000FFF1FBC1200200000FE2F000000207047704710B5FFF70DFE00F00BF800F04E
:20132000A7F810BD704710B5FFF7F8FD00F0E6F810BD0000014802490860704700366E01E7
:201340002800002007484068000C00040121C903401805490969084302494860C8030349E3
:201360008860704700100240000FFF1F00ED00E04022016A1140002915D0016849699201A8
:201380009143426A11430268516101221203416A914208D101684969032252039143826A79
:2013A000114302685161704700B587B000BF2F48406B012108432D4948630846406BC007EB
:2013C000C00F019000BF00BF00BF0846406B01210843264948630846406BC007C00F0190D0
:2013E00000BF00BF00BF0846C06B0121490408431E49C8630846C06B01214904084001902A
:2014000000BF00BF00BF194840300068C9100843164940310860084600680121890308404E
:20142000019000BF00BF042002900220039001200490022005900120069002A90520000738
:20144000FFF786FC022002900920069002A905200007FFF77DFC012200211C20FFF7BCFD2C
:201460001C20FFF7A7FD07B000BD00000010024010B5FFF799FF1D481D490860E120400207
:20148000486000211A488160C1600161816108214161FFF709FE174817490860E1204002A9
:2014A0004860002114488160C160016181610C214161FFF7F9FD10480068C068FF210131CC
:2014C00008430D490968C8600B48006840690121084309490968486107480068C068202175
:2014E000084305490968C86010BD0000003801401013002000440040BC12002010B50E48A4
:201500000068002816D00D480068401C0B490860084600680A280DD90948FFF79DFD09497F
:201520000860084601680648006800F077FA00200149086010BD000014000020180000206A
:20154000200000201C000020FEB5044620680069012149038843E1680843216808612169D8
:20156000A06808436169084302902068C0685E490840029908432168C860E06902902068D8
:2015800040690121C9028843029908432168486120684069032109028843A16908432168C9
:2015A00048610121C902E06988424ED1FFF724FD05466268510019226A431046FEF79AFD1C
:2015C00006466421FEF796FD07016268510019226A431046FEF78EFD06466268510019222F
:2015E0006A431046FEF786FD64210090FEF782FD64214843301AC00032300190FEF77AFD6E
:20160000F821084040003F186268510019226A431046FEF76FFD06466268510019226A43C9
:201620001046FEF767FD64210090FEF763FD64214843301AC00032300190FEF75BFD4007F0
:20164000400F3818216888604CE0FFF7D5FC05466268910019226A431046FEF74BFD06461A
:201660006421FEF747FD07016268910019226A431046FEF73FFD06466268910019226A434B
:201680001046FEF737FD64210090FEF733FD64214843301A000132300190FEF72BFDF02115
:2016A00008403F186268910019226A431046FEF721FD06466268910019226A431046FEF705
:2016C00019FD64210090FEF715FD64214843301A000132300190FEF70DFD0007000F381825
:2016E00021688860FEBD0000F3E9FFFFFFB581B004460D4617460A9E24E0701C002821D0B4
:20170000002E05D0FFF7FEFB0499401AB04219D92068C068FF21A13188432168C860206856
:201720004069400840002168486120214D2001554E20015500BF00214C20015500BF0320FA
:2017400005B0F0BD206800682840A84201D1012000E00020B842D0D00020F1E710B500F0AB
:2017600001F810BD10B50548FFF784FC00200449086001200349086010BD0000BC120020B6
:2017800018000020140000200FB410B503A9044B044A029800F062F810BC08BC04B0184785
:2017A000AD1900083C00002030B47446641E2578641CAB4204D3635D5B00E31830BC18479D
:2017C0001D46F8E710B5002819DB1A4A03231B02D21883089B00D2588307DC0EFF23A3408C
:2017E0009A438B071B0E8407E40EA3401A43114B032424021B198408A4001A5118E00E4ACC
:2018000003071B0F083B9B089B00D2588307DC0EFF23A3409A438B071B0E8407E40EA34078
:201820001A43054B0407240F083CA408A4001A5110BD000000E100E01CED00E002E008C895
:20184000121F08C1002AFAD170477047002001E001C1121F002AFBD170470000FFB58DB099
:201860000446002506E025280AD0109A0F999047641C6D1C20780028F5D1284611B0F0BD58
:2018800000270121484A009700E00743641C23780846203B98401042F7D120782E2817D120
:2018A000042007436078641C2A280CD10E98641C02C800910E900BE000990A225143303967
:2018C0004018641C00902078014630390929F3D920780028D1D0642808D0692806D0752891
:2018E0001ED0109A0F9990476D1C5BE00A200E99019001C90E91002802DA40422D2102E08C
:20190000390504D52B216A461172012103E0F90704D02021F7E70BAE0B910DE00021FAE7F5
:201920000A200E99019001C90E91F7E70199FEF7E1FB3031761E31700028F7D103A8801BC7
:2019400020300190780701D5009801E0012000900199884201DD401A00E0002000270090D4
:2019600006E002A8109AC05D0F9990476D1C7F1C0B988742F5DB04E0109A30200F999047D4
:201980006D1C0099481E00900029F5DC05E03078109A761C0F9990476D1C0199481E0190D3
:2019A0000029F4DC641C65E70928010013B50C46034B012269460348FFF7BCFB00981CBD8D
:2019C000FFFF0000101300200025002601270024FFF7A0FC1048FFF7EBF805463D4000BFE5
:2019E00008E00120A0402840002801D1274603E0601CC4B2012CF4DB00BF0748FFF7D8F88A
:201A00000646012E03D100213846FFF715FC01E0FEF730FEFCE7000000AF000870B50546C3
:201A20000C46224629460348FEF77AFB0248046070BD0000281200201000002070B50446F4
:201A40000D467D23DB002A4621460248FFF772FB70BD0000101300200000000000000000C4
:201A6000000000000000000000000000000000000000000000000000010000000200000063
:201A8000030000000400000006000000070000000800000009000000000000000000000021
:201AA000000000000000000001000000020000000300000004000000D81A00080000002002
:201AC000400000003C180008181B000840000020401500004C18000800000000000000000E
:201AE0000020000800000000000000000000000000000000000000000000000000000000BE
:201B000000127A000000000004000000010000000000000000000000FFFFFFFFFFFFFFFF3C
:201B2000FFFFFFFFFFFFFFFFFFFFFFFFFFFFFFFFFFFFFFFFFFFFFFFFFFFFFFFFFFFFFFFFC5
:201B4000FFFFFFFFFFFFFFFFFFFFFFFFFFFFFFFFFFFFFFFFFFFFFFFFFFFFFFFFFFFFFFFFA5
:201B6000FFFFFFFFFFFFFFFFFFFFFFFFFFFFFFFFFFFFFFFFFFFFFFFFFFFFFFFFFFFFFFFF85
:201B8000FFFFFFFFFFFFFFFFFFFFFFFFFFFFFFFFFFFFFFFFFFFFFFFFFFFFFFFFFFFFFFFF65
:10200000F0150020D5200008B56600081B5D00080B
:1020100000000000000000000000000000000000C0
:10202000000000000000000000000000C77600086B
:102030000000000000000000E5690008C178000809
:10204000E7200008E7200008E7200008E720000854
:10205000E7200008E7200008E7200008CD37000847
:1020600000000000E720000809360008000000001A
:10207000E7200008E7200008E72000080000000033
:10208000E7200008E720000800000000E720000823
:1020900000000000E7200008E7200008E720000813
:1020A0000000000015730008E7200008E720000882
:1020B000457D0008E7200008E72000080000000038
:1020C0000348854600F0AEF900480047D98A000869
:1020D000F01500200448804704480047FEE7FEE76B
:1020E000FEE7FEE7FEE7FEE7E5780008C12000080E
:1020F00030B50B46014600202022012409E00D46A0
:10210000D5409D4205D31D469540491B2546954027
:1021100040191546521E002DF1DC30BD70B500246B
:102120002546002801DA01244042002901DA012570
:102130004942FFF7DDFFAC4200D04042002C00D006
:10214000494270BD03460B439B0703D009E008C911
:10215000121F08C0042AFAD203E00B780370401C57
:10216000491C521EF9D27047D2B201E00270401CE5
:10217000491EFBD270470022F6E710B513460A4607
:1021800004461946FFF7F0FF204610BD421C0178B7
:10219000401C0029FBD1801A70470321001D401EFE
:1021A000037812021A43491EF9D510467047F8B554
:1021B00002464A40D40F42004B0052085B089A4244
:1021C00002D20246084611464A0023D0C30D4A00F7
:1021D000DDB2120EAD1A202D35DA49020126490A68
:1021E000F6058A19002C00D0524220214F1B1146BF
:1021F000B9402A411018C20D9A4221D0002C17D0A4
:10220000012D08DCDA05801AD20F8019D207DBB263
:1022100000F0CFF8F8BDDA05801A012340001B0654
:10222000C01880185A428018CA0F1043490007E0AE
:102230004908C2071143DA05801A8019400880183E
:1022400000F0AFF8F8BD61000122511A001BF7E75A
:102250000122D2075140AAE70122D2075040A6E747
:10226000024670B54A40D30FDB0740002DD04A002C
:102270002AD0010E140E000212020919400A520A55
:102280008418E50104465443000A120A2E04504300
:10229000A4194219200CC543AA18120C0125AD033C
:1022A000521C521912047F39240400D0521C1043CE
:1022B00001D44000491EC2B20C06C0092018401CBF
:1022C0004008802A02D003E0002070BD4008400092
:1022D000002900DA0020184370BD70B502464A405C
:1022E000D50F40004A00ED0740085208002814D0DE
:1022F000002A12D0C40DD30D41020120C0055202A4
:10230000490A520AE41A091812187D34914201D37D
:10231000641C00E04900002C01DA002070BD00239D
:10232000914201D3891A0343400849000028F7D19C
:1023300000290AD0914202D10121C90705E091424A
:1023400001D2012101E00121C943E005C018401973
:1023500000F027F870BDC217C10F504010B54018EB
:10236000CA079623002100F024F810BD10B5002202
:102370009623114600F01DF810BD410040020122D5
:10238000400AD205090E80187F2901DA0020704723
:10239000962903DC9622511AC84070479639884026
:1023A0007047002904DA401C490001D14008400070
:1023B000704770B40024050C05D11024000402D12C
:1023C000002921D01124050E01D100020834050F87
:1023D00001D10001241D850F01D18000A41C00281B
:1023E00001DB4000641C002908D020252E1B0D466F
:1023F000F540A14000D001212943084301061B1BE1
:10240000000ADB1D02D5002070BC7047DB051818E0
:1024100080180029F8DA401C4900F5D170BC40084A
:1024200040007047064C0125064E05E0E36807CCE6
:102430002B430C3C98471034B442F7D3FFF744FECB
:102440006C9B00088C9B000870B58C180578401CAC
:102450006B075B0F01D10378401C2A1106D102786B
:10246000401C03E006780E70401C491C5B1EF9D12D
:102470002B0705D40023521E0DD40B70491CFAE71C
:102480000378401CCB1A921C03E01D780D70491C88
:102490005B1C521EF9D5A142D8D3002070BD0000AC
:1024A000F8B505460E4617461C4601200649087039
:1024B00002F026F9054801F003FB02F0D5F80020F0
:1024C000208003490860F8BDC800002000AD000866
:1024D0004402002030B504460120034D287000203E
:1024E0001880024D286030BD4802002044020020C0
:1024F0001FB504461148007800281DD1FD2168460B
:102500000170FC214170FB218170FA21C17004210E
:10251000017100214171F02181710021C1710472AA
:102520004172042181720321C172022101730121D0
:1025300041730E2106F06CFF1FBD0000C900002092
:1025400038B504460020009020688068C007C00F9E
:10255000012148404840002827D12068806814495C
:102560000840002801D1012000E00020002809D106
:10257000A06B10210843A063E06B01210843E063D6
:10258000012038BD206880680121084321688860E7
:10259000084909480068FFF7ABFD009002E0009889
:1025A000401E009000980028F9D10020E9E70000C3
:1025B0001500008040420F0084040020F7B58AB067
:1025C000884800888749C9784843800008300B99BB
:1025D000884202DD84A005F019FC0024FAE0874857
:1025E0000990400C089040420790400C0690002053
:1025F000059004900025AAE07A48008860434019BD
:1026000081000A98405E0390764800886043691C08
:10261000401881000A98465E724800886043A91CF1
:10262000401881000A98405E02906E48008860431E
:10263000E91C401881000A98405E01900399891BAB
:1026400008B205F0F5FC07460299891B08B205F0AF
:10265000EFFC3F18019A0299891A08B205F0E8FCCC
:10266000381800B20090039805F0E2FC64498842F3
:1026700002DD0820059012E062490098884202DDE0
:10268000082005900BE009990398884201DD039822
:10269000099008990398884201DA039808905148F4
:1026A00000886043401981000A9808180221415EA1
:1026B00003914C4800886043691C401881000A98C7
:1026C00008180226865F474800886043A91C401806
:1026D00081000A9808180221415E02914148008851
:1026E0006043E91C401881000A9808180221415EE5
:1026F00001910399891B08B205F09AFC07460299DB
:10270000891B08B205F094FC3F18019A0299891AB6
:1027100008B205F08DFC381800B20090304605F084
:1027200087FC3749884202DD082004900EE03549D5
:102730000098884202DD0820049007E0079886424E
:1027400000DD07960698864200DA06966D1C25483D
:102750000088C01EA84200DD4EE70598072805DD69
:10276000032162000C980C30815412E001216200B8
:102770000C980C308154089A0999891808B205F010
:1027800057FC0746C00FC019401001B2A2000C98B8
:1027900081520498072806DD03226100491C0C9829
:1027A0000C30425415E001226100491C0C980C3099
:1027B0004254069A0799891808B205F039FC074671
:1027C000C00FC019401001B26000401C42000C98BC
:1027D0008152641C0348C078A04200DDFFE60DB0C2
:1027E000F0BD00009C04002052414D5F53495A4502
:1027F0005F6572725F6F70740A0000000180FFFFF6
:10280000204E0000B80B00001FB500200190029080
:1028100003902E48006B0121090508432B490863EA
:102820000846006B0121090588432849086300BF59
:1028300026484030006801210905084323494031FA
:10284000086008460068012109050840009000BFA3
:1028500000BF1F481F490860084601F077FA0028AA
:1028600001D000F039F81A481A4908600120000721
:102870004860002117488160C16001210161042185
:1028800041610121017600218176C176FF21C231AB
:10289000C161002101622430017024388162052168
:1028A000C16201F07BFB002801D000F015F8032085
:1028B000019001200003029001A9064801F0A8FA46
:1028C000002801D000F008F81FBD000000100240F1
:1028D00000240140840B002000BFFEE7002028E018
:1028E0008100154A51588200144B9A58914204D9DC
:1028F0008100114A5158820099508100104A515864
:102900008200104B9A58914204D981000C4A5158C8
:10291000820099508100084A515882000A4B9A5807
:10292000914204D909490978491C084A1170411C8F
:10293000C8B21028D4DB7047900F00201C0500207F
:10294000501000205C050020AC9A0008C000002058
:10295000F8B5164600241AE0A1001F4A8918022083
:10296000085E05F065FB0746A1001B4A505E05F0B6
:102970005FFB3946009000F03DFF054660001749B7
:10298000095AA94202DA600014490D52641C102C45
:10299000E2DB072E04D112480078401C1049087071
:1029A0000F480078042815DD00200D490870042424
:1029B0000DE060000949085A642807DD0120094933
:1029C0000870A00020180849088002E0641C082C48
:1029D000EFDB00BFF8BD0000E4050020E4060020A6
:1029E000CA000020AC040020AE040020F8B5054663
:1029F0000E4617460024002F0DD1002042490870D2
:102A0000424908704249088008460488102141481C
:102A1000FFF7B1FB75E0002D36D03B49097849003E
:102A20003C4A555238490978491CC9B2364A117096
:102A30000846C917490F0918C910C900411A117071
:102A400032480078082801DB082005E02F4800788C
:102A5000401CC0B22D4908702C490870002006E0C7
:102A600041002C4A515A09198CB2411CC8B227495D
:102A700009788842F4DB254801782046FFF74EFBB1
:102A800084B2234804803CE0002D38D1002E36D09B
:102A90001D49097849001F4A56521B490978491CAB
:102AA000C9B2194A11700846C917490F0918C91047
:102AB000C900411A117015480078082801DB082068
:102AC00005E012480078401CC0B2104908700F4958
:102AD0000870002006E041000E4A515A09198CB2D4
:102AE000411CC8B2094909788842F4DB07480178DB
:102AF0002046FFF713FB84B20548048001E0044838
:102B000004882046F8BD0000BD040020BE0400205B
:102B1000C0040020800D002010B50146114A00209D
:102B200016E083001B1DCB5C1C0283005B1DCB5C8D
:102B3000E3181BB2138083009B1DCB5C1C02830037
:102B4000DB1DCB5CE3181BB25380121D431C98B2F3
:102B5000054CA389DC17A40FE418A4108442E0DC20
:102B600010BD0000E40500201009002010B5044647
:102B70000020108002201880002010BDFEB5054600
:102B80000E46002409E029880C2060433B4A105877
:102B9000814200D108E0601C84B20C2060433749B8
:102BA000085837498842EED100BF0C2060433349B2
:102BB0000858334988425FD00C2060432F49085899
:102BC00075284BD00C2060430858712846D00C2043
:102BD00060430858702841D00C206043085874287E
:102BE0003CD0B01E81B20C206043244A80186B4652
:102BF000244A4768A81CB84701902A88684601887B
:102C00002048019B00F020FF1F4908800C206043F2
:102C10001A490858092804D00C20604308580A288B
:102C200002D10020184908800C206043134908583D
:102C300014281BD1154800780A2803DD0120144907
:102C4000087202E00020124908721248008800123F
:102C50000F4988720F480078C87207E00C20604363
:102C60000649401831468268284690470648018840
:102C70000748094A12689047FEBD000090020020F4
:102C8000FFFF00005208002038020020C000002092
:102C9000F8070020DE0000203C020020FFB581B0D4
:102CA00006460D4617462846E90F091849100091B7
:102CB00002200F49087000240EE06100705A03F0F2
:102CC00009FDA10078526100705A03F003FD000C69
:102CD000A100C9194880641C00988442EDD3009873
:102CE0008004010C04980180002005B0F0BD0000B4
:102CF000C600002010B5024804F0C8FA10BD00005C
:102D00001194000810B506F067FB0748006800281A
:102D100008D00548008881B2044800F009F8002076
:102D20000149086010BD0000E000002004070020F9
:102D300070B504460E460025002C01D0002E00D1AF
:102D400070BD0025A5E05548007C030005F06EF835
:102D50000B07121F2C393F5265727F8C9A00605D01
:102D60004F490978884204D100214C484182012111
:102D700001748BE0605D4A494978884203D10221A1
:102D80004648017402E00021444801747EE0605D21
:102D900043498978884203D103214048017402E005
:102DA00000213E48017471E0605D3D49C978884268
:102DB00003D104213948017402E00021374801742D
:102DC00064E0615D35488182052101745EE033482D
:102DD000808A615D0902401881B230488182808A10
:102DE000502803DC06212D48017402E000212B4805
:102DF00001744BE0615D2948428A408A401C83B2DD
:102E000026484382403881544030418A808A81423A
:102E100002D107212148017438E0605D2149097819
:102E2000884203D108211D48017402E000211B489B
:102E300001742BE0605D1B494978884203D1092168
:102E40001648017402E00021144801741EE0605D20
:102E500014498978884203D10A211048017402E09C
:102E600000210E48017411E0605D0E49C978884266
:102E700004D10A48818A4038FFF780FE00210748C4
:102E8000017403E000210548017400BF00BF681C05
:102E900085B2B54200DA56E700BF51E7E2070020ED
:102EA0003002002034020020F8B516461F460025E7
:102EB0003546012003F00EFC401CC4B2042003F090
:102EC00009FC80B20090601E28706870002008E045
:102ED0000121420052199170002142005219D17013
:102EE000401CA042F4D361004919009888700098F2
:102EF0000004000E61004919C8706000001D388090
:102F00000020F8BD70B504460D460E4801781F2913
:102F100004DA48000C4E305A108002E00020C04312
:102F2000108008488178042904DA4800064E305A97
:102F3000508002E00020C043508004201880002010
:102F400070BD000000BB00084A020020FFB581B040
:102F500006460D4617462846E90F09184910009104
:102F600000240EE06100705A03F0B4FBA100785217
:102F70006100705A03F0AEFB000CA100C919488033
:102F8000641C00988442EDD300988004010C0498DE
:102F90000180002005B0F0BDFFB585B005460F46A5
:102FA00000200490002600240390402002902888EE
:102FB0000290B81EC10F0918C9030E0C192E03DDAB
:102FC00000260120049016E007980390002410E0EA
:102FD00000210191621C5200A95C029AD0B201AAA0
:102FE00006F0ECF868468188620003988152601C04
:102FF00084B2B442ECDB7004010C089801800498A0
:1030000009B0F0BDF8B514461D4600F0FDF904F016
:1030100085FC064604F082FC871C222239462046A5
:10302000FFF790F87088801C28800020F8BD000011
:10303000F8B514461D460AA63046FFF7A7F82080CB
:103040003046FFF7A3F807463A463146A01CFFF783
:1030500079F83046FFF79AF8801C28800020F8BDE8
:1030600076332E322E300000F8B505460E46174650
:103070001C4600F08DF900202080F8BDFFB583B01C
:1030800005460E4617463046F10F091849100291C1
:10309000F520C0011549088028880190A888009073
:1030A00013490198087013490098087001201249CB
:1030B000087000240EE06100685A03F00BFBA100C9
:1030C00078526100685A03F005FB000CA100C91991
:1030D0004880641C02988442EDD302988004010C5D
:1030E00006980180002007B0F0BD0000C20000205B
:1030F000C4000020C5000020C600002030B50446F2
:103100000220108020205080042018800120024DD1
:103110002860002030BD000044020020F8B50546BC
:103120000E4617461C4604F047FE00F0A7FA0020A2
:10313000208001490860F8BD44020020FFB583B03B
:1031400006460F46002002900190002400250090C2
:1031500006213846FEF7CCFF019000BF1AE006209A
:10316000604385196878297800020843002806D151
:10317000A81CFFF712F800B20B49088002E00120FA
:10318000029000BF00BF0098002801D001200290EB
:10319000601C84B201988442E1DB00210698018022
:1031A000029807B0F0BD000042020020FFB583B0D6
:1031B00006460F46002406213846FEF799FF029086
:1031C00000252FE0062068438419607821780002EA
:1031D000084300280FD10120207000206070A01C3F
:1031E000FEF7DBFF0190617822780902114308465F
:1031F000019903F0F3FA607821780002084301286E
:103200000FD10420207000206070A01CFEF7C5FFC5
:10321000019061782278090211430846019903F070
:10322000DDFA6D1C02988542CCD300F0B1F8002184
:1032300006980180002007B0F0BD0000FFB583B004
:1032400006460F46002506213846FEF751FF02903C
:1032500000240FE0062060438519A81CFEF79DFF9F
:10326000019069782A78090211430846019903F010
:10327000B5FA641C02988442ECD30120034908701B
:10328000002106980180002007B0F0BDB0040020A6
:10329000FFB585B005460F46002004900390002638
:1032A00002900024019028880490B81E8003000C2E
:1032B000039000BF16E0B100A81C0C1862882178AA
:1032C000049BD8B205F088FF217801AA402005F0C0
:1032D00075FF608869468988884201D00120029084
:1032E000701C86B203988642E5DB002108980180B5
:1032F000029809B0F0BD10B504460020188010BD3A
:10330000F8B504460F461D462688A11C304604F039
:1033100009FB01200249087000202880F8BD000048
:103320004002002010B50024241D03F055FB0A497B
:10333000886003F055FB08494860084680880019FA
:1033400084B2802C02D905A004F060FD00F026F8BC
:1033500004F0BAF910BD0000600700204572726FDA
:10336000723A20666C617368446174614C656E20CA
:103370006973206D6F7265207468616E20464C41E0
:1033800053485F504147455F53495A45210D0A0054
:103390000120014908707047E4000020F8B50024BE
:1033A000002600270F4D00200090286800900E494D
:1033B0000098884204D00DA004F028FD00F0C2F867
:1033C00003F00EFB8003060C03F006FB0746002407
:1033D00005E02868A10078502D1D601C84B2B4421D
:1033E000F7DBF8BD00AC000879563412666C6173E7
:1033F000682073657474696E6720697320656D70E9
:103400007479210D0A00000030B500201249002215
:1034100000230A68091D114CA2420CD00824104D4B
:103420006C8000BF04E046250D4C241D2554401C33
:103430000828F8D30EE00B68091D1CB2084D6C80FB
:10344000002005E00D68064C241D2550091D001DB7
:103450002028F7D330BD000000AE00085555AAAAB9
:103460006C07002010B51E48007800280BD000F033
:1034700089FB00F089F800201949087003F01CF955
:1034800000201849087018480078002804D000F07F
:1034900031F800201449087014480078002812D030
:1034A00012480078032805DA10480078401C0F49BC
:1034B000087008E00D480078032804D100F090F867
:1034C00000200A4908700A480078002800D110BD81
:1034D00000F038F800200649087000BFF7E7000048
:1034E000400200206C04002048020020410200201D
:1034F000E40000201CB5104C002001900090012039
:10350000009001F0FDF8204600F0DAFA0B48019037
:10351000012201A9204600F007FB241D0122694673
:10352000204600F001FB241D20220549204600F022
:10353000FBFA01F099F81CBD00AD00085555AAAA88
:10354000C700002070B503F047FA044603F048FABC
:10355000054601F0D5F80B4800F0B2FA0948803072
:1035600000F0AEFA22460749012001F08FF822460A
:10357000803204498031012001F088F801F074F8AC
:1035800070BD000000AC00081CB5124C002001907A
:10359000009011480221415E009101F0B1F82046EF
:1035A00000F08EFA0D480190012201A9204600F09A
:1035B000BBFA241D01226946204600F0B5FA241DFD
:1035C00020220549091D204600F0AEFA01F04CF812
:1035D0001CBD000000AE00086C0700205555AAAACB
:1035E00010B5074C01F08CF8204600F069FA09226A
:1035F0000449204600F098FA01F036F810BD0000AA
:1036000000BB00089007002010B50249886D00F04B
:1036100083FE10BD8009002030B50124056CAC404C
:10362000C56B6C60046863604468102C04D1046846
:10363000A2600468E16003E00468A1600468E260DD
:1036400030BD000010B50E210A48FEF794FD082198
:103650000948FEF790FD084800F0A8FA064840889F
:10366000083804498881044949884904080C03F052
:1036700073FF10BD100900206004002010B50E215A
:103680000B48FEF778FD08210A48FEF774FD03F0A9
:10369000DFFE084800F08AFA0648408808380449E6
:1036A0008881044949884904080C03F055FF10BD7E
:1036B000100900206004002010B50446204600F0E8
:1036C00045FF10BDF8B504460E46002000900025C9
:1036D00002F03CFF002802D00220009000E001250B
:1036E00020882B460422694602F022FE0149088008
:1036F0002846F8BD38020020F8B504460F460020E1
:1037000000900326002502F021FF002809D00A4876
:1037100000F034FA064600960098C007C00F0090EB
:1037200000E0012520882B460422694602F000FEB5
:10373000024908802846F8BD00AF00083802002082
:10374000F8B504460F46002600200090002502F040
:10375000FDFE002804D001F04DF90646009600E079
:10376000012520882B460422694602F0E1FD284607
:10377000F8BD000070B504460E46012502F0E6FED5
:10378000002811D00D4800F09BF9322000F0DEFE39
:1037900000BFBFF34F8F0A480A49C860BFF34F8F7D
:1037A00000BF00BF00BFFDE720882B460022114666
:1037B00002F0BEFD04490880284670BD00AF000835
:1037C0000400FA0500ED00E038020020402008491E
:1037D000C9680140814201D1012100E00021002996
:1037E00004D040200249C86000BF00BF70470000FD
:1037F0000018024070B502468A4201DB154600E01F
:103800000D462B468A4201DA154600E00D462C464D
:103810005D115E1B0B2565436D117519A8B270BD56
:1038200070B502468A4201D3154600E00D462B468C
:103830008A4201D2154600E00D462C465D095E1B0A
:103840000B2565436D09701970BD000000B500209F
:103850000649486000F054FF0548406904210843C8
:10386000034948610348C106086000BDD00B002031
:10387000002002402143341200B5034600200D49C8
:10388000486000F03DFF0C484069022108430A49A6
:103890004861FF20186000BF074800690121090442
:1038A0000840002805D004480069C007C00F002860
:1038B000F2D000BDD00B002000200240F0B5A9B02E
:1038C00004460F460020289027902690002525903A
:1038D000219022902390249000260090A007800F32
:1038E000002802D0681E29B0F0BD1F48844203D8CA
:1038F0000120C006844202D20020C043F3E7012029
:10390000C006201A28902898C00926902698C00141
:103910000121C9064518601B27900095002604E088
:103920000098805D01A98855761C802EF8D302206E
:10393000219022950120249025A921A800F01CFEA9
:10394000002802D00020C043CDE701A927980F50DE
:1039500001AA2946012000F099FE002802D000208B
:10396000C043C0E70020BEE700C00008F0B5024633
:103970000B46002014461D46144E766901273E432F
:10398000124F7E6100BFEFF31086314672B60EE033
:103990002E6826602D1D241D461CF0B21F2806D15E
:1039A0000A4E76690127FF043E43084F7E612028B6
:1039B000EED300BF054E366901273F043E40002E7E
:1039C000F8D100BF81F3108800BFF0BD0020024095
:1039D00000B5034600F094FE0B4840690121C9027E
:1039E000084309494861FF20186000BF0648006984
:1039F000012109040840002805D003480069C007D8
:103A0000C00F0028F2D000BD0020024070B504466F
:103A100000F0EAFF051905E000F0E6FFA84201D337
:103A2000032070BD06480069012109040840000C0C
:103A30000028F1D10348024908610020F1E70000A5
:103A40000020024011800000FFB581B006460D46FF
:103A5000174600244E2D02DD002005B0F0BD1549AB
:103A6000081904221449FEF76DFB201D84B2281D9D
:103A700010490853A01C84B2FF200130384308537A
:103A8000A01C84B204980853A01C84B2002E06D057
:103A900008192A463146FEF755FB601984B20549DC
:103AA000081904220549FEF74DFB201D84B220466B
:103AB000D3E70000F8070020300200203402002085
:103AC00010B586B00446002001906006400E002824
:103AD00003D00020C04306B010BD02200290039422
:103AE0000120059001A902A800F046FD002803D09E
:103AF00002A0019904F08AF90020ECE748414C5FEC
:103B0000464C41534845785F457261736520457264
:103B1000726F722C506167654572726F72203D2022
:103B200025640D0A00000000F8B504460F4615464E
:103B30000026A80000191049884201D9701EF8BD5E
:103B4000A007800F002802D00020C043F7E700261E
:103B50000DE0B00039582046FFF7B0FE002801D133
:103B6000241D02E00020C043E9E7701C86B2AE428B
:103B7000EFDB0020E3E7000000C000080146086812
:103B80007047000010B507480068012808D103F00D
:103B900051FA02F091FD00200349086001490860D4
:103BA00010BD0000500400205804002010B5044649
:103BB000002C01D1401E10BD03F06AFA207020785D
:103BC00000280BD001280FD0022810D0032813D1D1
:103BD00003F0AEFA80000830608013E003F092FA40
:103BE0008000083060800DE0094860800AE003F042
:103BF0007CFA0830608005E006A004F007F9002098
:103C0000C043D8E700BF03F088FAA0800020D2E7C5
:103C1000081000004572726F723A20756E737570ED
:103C2000706F72742064617461547970650D0A005C
:103C3000F0B585B004460D4600200490002703909F
:103C400002F0CAFE029002998868FEF78FFB39499C
:103C50000090FEF705FB0190FEF78FFB36490860E8
:103C600036480078012807D108460068401C3449CE
:103C70000860002031490870002C01DC002D00DDB7
:103C80000127012F09D12F48007806280EDA2D4888
:103C90000078401D2B49087008E02A480078002869
:103CA00004DD28480078401E264908702548007821
:103CB000052802DD0120039001E00020039000268A
:103CC0000398012804D1049000201D4908602EE0CB
:103CD0001D480078012810DB19480068164909685A
:103CE000884205D30020049015490860012604E0AD
:103CF000012F02D1002012490860012E17D0104870
:103D000000680D490968884204D3002004900C49DA
:103D100008600CE0022004900948006801210905B0
:103D2000884204D206480068401C0549086004988F
:103D300005B0F0BD0000D040A8040020B004002071
:103D4000B8040020BC040020D6000020F8B50446CA
:103D500000250026002700BF3420005D012801D186
:103D60000220F8BD01213420015500BF2068806881
:103D700008404840484000283ED1A06B09028843D3
:103D800002210843A0632068C0688707BF0F20682E
:103D9000C068800880002168C860206880680121B0
:103DA000C90708432168886000F01EFE064611E03E
:103DB00000F01AFE801B02280CD9A06B0221884358
:103DC00010210843A06300BF00213420015500BF2B
:103DD0000120C6E720688068C00FC0070028E7D12F
:103DE0002068C06838432168C860A06B02218843FE
:103DF00001210843A06304E0A06B20210843A063D5
:103E0000012500BF00213420015500BF2846A8E746
:103E1000F8B504460D46002600200090E06A002810
:103E200015D0E06A012812D0E06A02280FD0E06ABB
:103E300003280CD0E06A042809D0E06A052806D0DF
:103E4000E06A062803D0E06A072800D000BF00BF60
:103E50003420005D012801D10220F8BD0121342069
:103E6000015500BF206880680421084080080028B0
:103E70007BD14449686888425AD02068806A2A7891
:103E800001219140084321688862E06A002829D016
:103E9000E06A012826D0E06A022823D0E06A0328DD
:103EA00020D0E06A04281DD0E06A05281AD0E06A14
:103EB000062817D0E06A072814D0A8682168496945
:103EC0004907490F88420DD020684069C008C000EA
:103ED0002168486120684069297A4907490F0843E9
:103EE0002168486128680B2802D028680C2841D135
:103EF0002548806829680B2902D10121C90501E004
:103F00000121890508432049886028680B2831D1A0
:103F10001E491F480068FEF7EBF80A21484300904D
:103F200002E00098401E009000980028F9D121E09E
:103F30002068806A2A78012191408843216888623C
:103F400028680B2802D028680C2813D10E488068F6
:103F500029680B2903D10121C90502E005E00121EF
:103F6000890588430849886004E0A06B2021084344
:103F7000A063012600BF00213420015500BF304658
:103F80006BE70000011000000027014040420F00D5
:103F90008404002001460868006C704770B5044630
:103FA00000260025002C01D1012070BDA06B002847
:103FB00006D1E063002134200155204600F0C0F80E
:103FC000A06B1021084000287ED1002EFCD1206873
:103FD00080680421084080080028F5D1A06B890181
:103FE000884302210843A06320688068C007C00F8F
:103FF00001214840484000280FD12068C06818219E
:104000008843A16808432168C860206800690001EE
:10401000000961680843216808612068C068464952
:1040200008402168C860207E8003617EC903084380
:10403000A17E49030843A16A012902D00121090395
:1040400000E000210843E16808432169022901D109
:10405000042100E0002108432421095D49000843B0
:104060000543E07E01280ED1A07E002803D1012067
:104070000004054307E0A06B20210843A063E06B28
:1040800001210843E063FF21C231E069884203D087
:10409000216AE069084305432068C0682843216815
:1040A000C860E06A002816D0E06A012813D0E06AF0
:1040B000022810D0E06A03280DD0E06A04280AD054
:1040C000E06A052807D000E02EE0E06A062802D06A
:1040D000E06A07280DD120684069C008C000216847
:1040E000486120684069A18D4907490F084321684C
:1040F00048612068C06811490840A84208D10020E2
:10410000E063A06B0221884301210843A06310E013
:10411000A06B0221884310210843A063E06B0121BA
:104120000843E063012604E0A06B10210843A0636C
:104130000126304639E7000019C2FEFFE7FF3F8342
:104140007047F8B504460D466069022801D108277A
:1041500011E02068C068C007C00F00280AD0A06B1B
:1041600020210843A06300BF00213420015500BF77
:104170000120F8BD0C2700F037FC064614E0681C4F
:10418000002811D0002D04D000F02EFC801BA84286
:104190000AD9A06B04210843A06300BF002134208A
:1041A000015500BF0320E4E720680068384000287C
:1041B000E5D0A06B012149020843A0632068C068D4
:1041C000032189020840002825D1A07E002822D1A1
:1041D000206800680821084008281CD120688068F1
:1041E00004210840800800280DD1206840680C2177
:1041F000884321684860A06BFF2101318843012179
:104200000843A06307E0A06B20210843A063E06B94
:1042100001210843E063207E002802D10C202168A0
:1042200008600020A5E7000070B50446002520685E
:10423000806804210840800800282BD100BF34206A
:10424000005D012801D1022070BD012134200155FB
:1042500000BF607E012803D02046FEF771F90546B5
:10426000002D18D1A06B0D490840FF2101310843F2
:10427000A0630020E06300BF00213420015500BF8F
:104280001C20216808602068806804210843216898
:10429000886000E002252846D6E70000FEF1FFFF17
:1042A00070B5044600252120005D022803D00420BB
:1042B000A06301252BE0206800680E218843216857
:1042C00008602068006840084000216808601149C3
:1042D0002068884201D1012008E00E49143120688D
:1042E000884201D1102001E0FF200130094908393E
:1042F000486001212120015500BF002120200155E7
:1043000000BF606B002802D02046616B88472846BA
:1043100070BD00000800024070B50446E06B0568FF
:10432000206806680420216C88402840002828D096
:1043300004203040002824D0206800682021084054
:10434000002805D12068006804218843216808609E
:104350003A492068884201D1042008E037491431E5
:104360002068884201D1402001E0012080023349C9
:1043700008394860E06A00285FD02046E16A884733
:104380005BE00220216C88402840002830D00220C9
:10439000304000282CD020680068202108400028E8
:1043A00008D1206800680A2188432168086001213B
:1043B0002120015521492068884201D1022008E0CE
:1043C0001E4914312068884201D1202001E00120DB
:1043D00040021A490839486000BF002120200155D9
:1043E00000BFA06A002828D02046A16A884724E0A0
:1043F0000820216C8840284000281ED0082030402A
:1044000000281AD0206800680E21884321680860BF
:104410000120216C8840E16B48600120A0630121EC
:104420002120015500BF00212020015500BF206B35
:10443000002802D02046216B884770BD080002404A
:1044400070B504460025002C01D1012070BD164A2C
:104450002168881A1421FDF74BFE80002064124861
:104460000838E063022121200155206805680F48C3
:104470000540A16860680843E16808432169084372
:1044800061690843A1690843E1690843054320685D
:1044900005600020A063012121200155002120207A
:1044A00001550020D2E70000080002400FC0FFFFC6
:1044B000F8B504460D4616461F460020009000BF82
:1044C0002020005D012801D10220F8BD012120201B
:1044D000015500BF2120005D01282DD1022121209E
:1044E00001550020A0632068006840084000216852
:1044F00008603B46324629462046FFF78DF8E06AC1
:10450000002806D0206800680E2108432168086052
:104510000BE0206800680421884321680860206857
:1045200000680A21084321680860206800680121AA
:1045300008432168086006E000BF002120200155E3
:1045400000BF022000900098BFE7000070B504464D
:1045500000F04AFA06462546681C002802D00548A5
:1045600000682D1800BF00F03FFA801BA842FAD364
:1045700070BD000090040020F8B504460E460127E7
:10458000002500BF36480078012801D10220F8BD7F
:1045900001203349087000BF2068012815D17D2013
:1045A000C000FFF733FA002852D1FFF74FF97D2002
:1045B000C000FFF72BFA074600F0A2F8294840692F
:1045C000042188432749486142E02068022825D118
:1045D0007D20C000FFF71AFA002839D1401E306054
:1045E000656814E02846FFF747F97D20C000FFF713
:1045F0000DFA074600F084F81A4840690221884302
:1046000018494861002F01D0356006E08035E06828
:10461000C00161684018A842E4D819E02068032866
:1046200016D17D20C000FFF7F1F9002810D1A06855
:10463000FFF7CEF97D20C000FFF7E8F9074600F04C
:104640005FF8084840690121C9028843054948616B
:1046500000BF00200249087000BF384697E70000FD
:10466000D00B002000200240012007494969C20701
:104670001143054A516111464969C90FC90700290B
:1046800000D000207047000000200240F8B5074627
:104690000D461646012400BF17480078012801D1B5
:1046A0000220F8BD01201449087000BF7D20C00021
:1046B000FFF7ACF90446002C16D100F021F8314682
:1046C0002846FFF753F97D20C000FFF79FF9044605
:1046D00000F016F809484069400840000749486161
:1046E000002C01D02046DCE700BF00200249087002
:1046F00000BF2046D5E70000D00B0020002002407C
:10470000002009494969C90FC90700290BD0074989
:10471000054A91600649916011464969C90FC90768
:10472000002900D001207047002002402301674586
:10473000AB89EFCDF0B502460B4600206AE00125BB
:10474000854029461940002963D0354D8608B600BA
:10475000AC598507EE0E0F25B5402C4005252D07D9
:10476000AA4201D1002505E02E4DAA4201D1012522
:1047700000E002258607F60EB540A54223D1284D5C
:1047800020352D688D43264E2036356035466D68C0
:104790008D437560224D603D2D688D43204E603EF7
:1047A000356035466D688D4375608507EE0E0F25C3
:1047B000B5402C461A4D8608B600AD59A543184E93
:1047C0008708BF00F551156847000326BE403543F2
:1047D0001560C508AE0015462035AD594607F70EE1
:1047E0000F26BE40B543C608B60017462037BD5158
:1047F000956847000326BE40B5439560556801267D
:104800008640B5435560D56847000326BE40B54392
:10481000D560401C1D46C540002D90D1F0BD000064
:10482000601802400004005070B503460022CBE03F
:10483000012696400C683440002C71D04D68022D42
:1048400002D04D68122D15D1D508AE001D46203579
:10485000A8595507EE0E0F25B5400646AE43304623
:104860005607F60E0D69B5402843D508AD001E4623
:1048700020367051186856000325B5400646AE43F1
:1048800030460D79AD07AD0F5600B540284318608E
:104890004D68012D08D04D68022D05D04D68112DB1
:1048A00002D04D68122D18D1986856000325B540E6
:1048B0000646AE4330465600CD68B5402843986062
:1048C0005868012595400646AE43304610264D688F
:1048D00035402D09954028435860D8685600032577
:1048E000B5400646AE43304656008D68B540284375
:1048F000D860012636074D683540B54263D1354D45
:104900009608B600A8599507EE0E0F25B540064645
:10491000AE43304605252D07AB4202D1002506E007
:1049200051E02D4DAB4201D1012500E00225960753
:10493000F60EB5402843274D9608B600A851254DE0
:10494000203528680546A5432846012636044D68CB
:104950003540B54202D10546254328461D4D203538
:10496000286068680546A5432846012676044D68F8
:104970003540B54202D1054625432846154D203520
:104980006860144D603D28680546A5432846012609
:1049900036054D683540B54202D1054625432846C7
:1049A0000C4D603D286068680546A54328460126F1
:1049B00076054D683540B54202D105462543284667
:1049C000044D603D6860521C0D68D540002D00D03C
:1049D0002EE770BD6018024000040050002A01D08C
:1049E000816100E081627047014800687047000003
:1049F000880400200148006870470000000EFF1F77
:104A000070B50446002C01D1012070BD3920005D35
:104A1000002805D1002138200155204600F01CFB5C
:104A20002421392001552068006840084000216891
:104A3000086000F01FFC054659496068884206D8A6
:104A40005848854201D2012007E0002005E0564881
:104A5000854201D2012000E00020012800D1D4E7E6
:104A600052492846FDF744FB064620684068810904
:104A7000890131432068416049496068884201D812
:104A8000701C08E0FF212D31714308467D21C900CB
:104A9000FDF72EFB401C2168096A8909890108433A
:104AA000216808623E496068884214D862685100F3
:104AB000681EFDF71DFB401C0005000D042801D2F7
:104AC000042041E062685100681EFDF711FB401CA4
:104AD0000005000D38E0A068002807D16268530087
:104AE000D118681EFDF704FB401C0AE01923626818
:104AF0005A431146681EFDF7FBFA401C0121890349
:104B000040180005000D002801D101201CE0A0681C
:104B1000002809D162685300D118681EFDF7E8FA31
:104B2000401C0005000D0CE0192362685A43114631
:104B3000681EFDF7DDFA401C0005000D0121890308
:104B400040180121C90308432168C969184A114066
:104B500008432168C861E169A069084321680968C0
:104B6000C022914308432168086020688068FE21C4
:104B70008843E16808432168886020680068012153
:104B80000843216808600020E06320213920015596
:104B90000020E06200213A200155002035E70000A6
:104BA000A086010080841E0000093D0040420F00E5
:104BB0000030FFFFFFB583B004460F460E9EFFF79F
:104BC00013FF05463920005D202877D119230122E3
:104BD000C1492046009501F067FA002802D0022062
:104BE00007B0F0BD00BF3820005D012801D10220D0
:104BF000F6E701213820015500BF20680068084011
:104C0000002804D1206800680843216808602068F3
:104C100000680121C90288432168086022213920E7
:104C2000015540213A2001550020E0630C98206294
:104C30000D98E084E08CA084A848A06200960195BD
:104C400039462046069B059A01F0D8F8002801D085
:104C50000120C5E7A08C002811D100BF0290206878
:104C60004069029020688069029000BF00BF206800
:104C700000680121490208432168086050E0A08CC7
:104C800001281CD12068006801218902884321681D
:104C9000086072B600BF0020029020684069029050
:104CA00020688069029000BF00BF20680068012171
:104CB000490208432168086062B631E009E1A08C2E
:104CC00002281BD1206800680121C902084321681D
:104CD000086072B600BF0020029020684069029010
:104CE00020688069029000BF00BF20680068012131
:104CF000890288432168086062B611E02068006874
:104D00000121890208432168086000BF0020029049
:104D100020684069029020688069029000BF00BF4F
:104D2000C7E0A08C032876D8A08C012816D12A468B
:104D30003146204601F060FA002801D001204FE7FB
:104D400020680069216A0870206A401C2062A08CDB
:104D5000401EA084E08C401EE084AAE0A08C0228C3
:104D60002ED1334600225E492046009501F09CF981
:104D7000002801D0012033E772B6206800680121C5
:104D8000490208432168086020680069216A0870A8
:104D9000206A401C2062A08C401EA084E08C401E33
:104DA000E08462B620680069216A0870206A401CAD
:104DB0002062A08C401EA084E08C401EE08478E03D
:104DC0003346002246492046009501F06DF900283F
:104DD00001D0012004E7206800680121890288438E
:104DE0002168086072B620680069216A0870206A2C
:104DF000401C2062A08C401EA084E08C401EE084F9
:104E00003346002236492046009501F04DF900282E
:104E100002D00120E4E622E0206800680121490276
:104E200008432168086020680069216A0870206AC8
:104E3000401C2062A08C401EA084E08C401EE084B8
:104E400062B620680069216A0870206A401C2062EE
:104E5000A08C401EA084E08C401EE08429E02A46FD
:104E60003146204601F0C8F9002801D00120B7E6FC
:104E700020680069216A0870206A401C2062A08CAA
:104E8000401EA084E08C401EE0842068406904211C
:104E90000840800800280CD020680069216A08704A
:104EA000206A401C2062A08C401EA084E08C401E22
:104EB000E084A08C002800D033E720213920015560
:104EC00000213A20015500BF3820015500BF0020C5
:104ED00086E6022084E60000020010000000FFFFCA
:104EE00004000100FFB583B004460F460E9EFFF795
:104EF0007BFD05463920005D20287DD11923012244
:104F000053492046009501F0CFF8002802D0022036
:104F100007B0F0BD00BF3820005D012801D102209C
:104F2000F6E701213820015500BF206800680840DD
:104F3000002804D1206800680843216808602068C0
:104F400000680121C90288432168086021213920B5
:104F5000015540213A2001550020E0630C98206261
:104F60000D98E084E08CA0843A48A06200960195F8
:104F700039462046069B059A00F0EAFF002801D03A
:104F80000120C5E736E02A463146204601F076F991
:104F900000280BD0E06B042806D1206800680121AE
:104FA00049020843216808600120B1E7206A0078BF
:104FB00021680861206A401C2062A08C401EA084E9
:104FC000E08C401EE084206840690421084080088D
:104FD00000280FD0A08C00280CD0206A007821680F
:104FE0000861206A401C2062A08C401EA084E08CD6
:104FF000401EE084A08C00E027E00028C3D12A46B0
:105000003146204601F01EF800280BD0E06B042842
:1050100006D1206800680121490208432168086020
:10502000012075E7206800680121490208432168D2
:10503000086020213920015500213A20015500BF88
:105040003820015500BF002062E7022060E7000021
:10505000020010000000FFFF10B586B004461421C6
:1050600001A8FDF788F800BF2748C06B012149055A
:1050700008432549C8630846C06B0121490508401B
:10508000009000BF00BF00BF1F48406B02210843D3
:105090001D4948630846406B02210840009000BF4C
:1050A00000BF00BF1848406B0843174948630846D3
:1050B000406B02210840009000BF00BF40200190DB
:1050C00012200290012003900220049006200590F7
:1050D00001A90E48FFF7A8FB80200190062005904B
:1050E00001A90A48FFF7A0FB0748C06A012149054A
:1050F00008430549C8620846C06A0121490588433A
:105100000149C86206B010BD001002400004005002
:1051100070B50446002C01D1012070BD0F482168F4
:1051200008600F482168086021686068486021684D
:10513000A0688860FFF758FC054606E0FFF754FCBE
:10514000401B302801D90320E7E72068C068002809
:10515000F4D10448216808600020DEE7CCCC0000D0
:1051600055550000AAAA0000014602480A681060CE
:1051700000207047AAAA0000034800680349096894
:1051800040180149086070478804002090040020FE
:1051900010B50024032000F009F8002801D00124F4
:1051A00001E000F033F8204610BD0000F8B50446D9
:1051B00000251348006800281ED0114801687D2092
:1051C000C000FCF795FF074639460E480068FCF71B
:1051D0008FFF064600F098FC00280BD1042C07D264
:1051E00000222146401E00F025F80748046004E034
:1051F000012502E0012500E001252846F8BD000058
:1052000090040020840400208C04002070470000DB
:105210000146002909DB00BF00BFCB06DB0E0122DF
:105220009A40034B1A6000BF00BF00BF70470000E8
:1052300000E100E070B504460D46164629462046BA
:1052400002F002FE70BD000000BFBFF34F8F0448A4
:105250000449C860BFF34F8F00BF00BF00BFFDE728
:105260000400FA0500ED00E0014800687047000006
:105270008404002000B5FFF7F7FF0649896807227C
:1052800012031140090B8900034A515CC906C90E7B
:10529000C84000BD001002400C99000810B504463B
:1052A000002C01D1012010BD02215D200155206894
:1052B00000684021884321680860204600F03EF9DC
:1052C0000020206600215D20015500BF5C200155B3
:1052D00000BF0020E7E7000010B50446216E02A0E1
:1052E00002F094FD10BD0000687370692D3E457298
:1052F000726F72436F6465203D20256420000000BA
:10530000F8B5044620684668206885684020284033
:10531000800900280FD1E807C00F0121484048400C
:10532000002808D0402030408009002803D02046C3
:10533000E16C8847F8BD022028404008002808D0CA
:1053400080203040C009002803D02046216D8847C6
:10535000F0E7202028404009002804D140202840C0
:10536000800900287DD0202030404009002878D0D6
:1053700040202840800900281ED05D20005D0328C1
:105380000ED0206E04210843206600BF002000904C
:105390002068C068009020688068009000BF0BE023
:1053A00000BF002000902068C068009020688068DE
:1053B000009000BF00BFBDE7202028404009002822
:1053C00011D0206E01210843206600BF002000900C
:1053D0002068806800902068006840218843216828
:1053E000086000BF00BF206E002839D020684068E8
:1053F000E02188432168486001215D200155022099
:105400003040002803D1F007C00F002825D02068C5
:1054100040688008800021684860A06D00280BD09B
:105420001148A16D4863A06DFEF73AFF002803D034
:10543000206E402108432066606D002810D00A4885
:10544000616D4863606DFEF72BFF002808D0206E69
:1054500040210843206603E003E02046FFF73CFFBD
:1054600068E700BF66E700002573000870B50446D2
:10547000002C01D1012070BD606A002800D100BF5E
:105480000021A1625D20005D002804D15C2001554F
:10549000204600F079F802215D200155206800685F
:1054A000402188432168086007210902E06888429A
:1054B00001D9002501E001252D030F210902E06833
:1054C000884206D007210902E068884201D0002105
:1054D000A162206B002809D107210902E0688842F7
:1054E00002D90221216301E001212163A1686068E2
:1054F0000843216908436169084301225202A169F6
:1055000011400843E1690843216A0843A16A08433E
:1055100021680860A069000C04210840616A084302
:10552000616B0843E1680843284321684860002014
:10553000206601215D20015500209CE710B504463E
:105540000F49206888421AD10E48006B891408431D
:105550000C4908630846006B8914884309490863AD
:10556000202105200007FFF7E5F84021052000076E
:10557000FFF7E0F8802105200007FFF7DBF810BDFA
:10558000003001400010024010B586B004466B495F
:10559000206888427ED100BF6948406B01210843E2
:1055A000674948630846406BC007C00F009000BFC2
:1055B00000BF00BF0846406B0121084360494863B3
:1055C0000846406BC007C00F009000BF00BF00BF7F
:1055D0000846406B01210843594948630846406B1F
:1055E000C007C00F009000BF00BF00BF0846406B5F
:1055F00001210843524948630846406BC007C00F69
:10560000009000BF00BF00BF4D48403000688914C3
:1056100008434B4940310860084600688914084037
:10562000009000BF00BF2020019002200290039054
:1056300004900020059001A905200007FFF7F4F869
:10564000402001900020059001A905200007FFF7E8
:10565000EBF8802001900020059001A905200007AB
:10566000FFF7E2F8102001900020059001A9052025
:105670000007FFF7D9F800BF3148806B01210843CC
:105680002F4988630846806BC007C00F009000BF99
:1056900000BF00E04FE000BF294840300068012112
:1056A000084327494031086008460068C007C00F1A
:1056B000009000BF00BF23482349086000204860D5
:1056C0000021214881608021C16007210902E06832
:1056D000884204D800211C480161416105E0FF2196
:1056E0000131194801618900416100211648816139
:1056F00001214903C161FEF7A3FE12481C38C069AD
:105700000321090388430F491C39C8610846C06951
:105710000321090308430B491C39C86100BF0A482B
:10572000A065446200BF012211460A20FFF782FDF6
:105730000A20FFF76DFD06B010BD000000300140EB
:10574000001002401C000240E4090020F8B50446A5
:105750000E46154600200090A06800280ED1FF21BB
:1057600005316068884209D104215D2001552B462E
:1057700032463146204600F0B7F8F8BD00BF5C2045
:10578000005D012801D10220F7E701215C200155CD
:1057900000BF5D20005D012802D0022000908AE059
:1057A000002E01D0002D02D10120009083E00421C1
:1057B0005D200155002020662664442005534620C4
:1057C00005530020E0642065A087E0874903A068B6
:1057D000884205D120680068491088432168086024
:1057E00007210902E068884207D920684068012142
:1057F000090388432168486024E02068406801214B
:105800000903084321684860A06D406901218902AD
:10581000884217D120684068890088432168486021
:105820004620005BC007C00F002805D14620005B62
:1058300041104620015305E04620005B4010401C0B
:10584000462108531F48A16DC8621F48A16D886298
:105850001E48A16D08630020A16D486346273B5B8D
:10586000276839460C31226CA06DFEF721FE002816
:1058700009D0206E102108432066012000900121EC
:105880005D20015517E0206800684021084040284D
:1058900004D02068006808432168086020684068D8
:1058A000202108432168486020684068012108439E
:1058B0002168486000BF00BF00215C20015500BF87
:1058C00000985AE765730008817300083D7300086B
:1058D0000121024A024B1B88D15470476C040020FE
:1058E0006E04002070470000F0B585B004460E46F7
:1058F00017461D460020019000BF5C20005D012876
:1059000002D1022005B0F0BD01215C20015500BF8D
:105910005D20005D029060680390029801280DD020
:10592000FF2105310398884205D1A068002802D1E3
:105930000298042802D002200190CAE0002E03D071
:10594000002F01D0002D02D101200190C1E05D2087
:10595000005D042802D005215D200155002020664D
:10596000A663A587E5872764442005534620055391
:105970000020E064206507210902E068884207D919
:10598000206840680121090388432168486037E0A6
:105990002068406801210903084321684860606D60
:1059A00040690121890288420CD1A08FC007C00F35
:1059B000002803D1E08F4010E08703E0E08F401023
:1059C000401CE087A06D406901218902884217D1FF
:1059D0002068406889008843216848604620005B51
:1059E000C007C00F002805D14620005B41104620AB
:1059F000015305E04620005B4010401C462108533F
:105A00005D20005D042806D13548A16DC862354887
:105A1000A16D886205E03448A16DC8623348A16D6C
:105A200088623348A16D08630020A16D4863462059
:105A3000035B206801460C31226CA06D0090FEF7DC
:105A400037FD002809D0206E102108432066012070
:105A5000019001215D2001553BE020684068012153
:105A60000843216848600020616DC862616D8862EA
:105A7000616D0863616D4863E38F206802460C32F4
:105A8000A16B606D0090FEF713FD002809D0206E19
:105A90001021084320660120019001215D2001555D
:105AA00017E02068006840210840402804D02068A2
:105AB0000068084321680860206840682021084386
:105AC00021684860206840680221084321684860D6
:105AD00000BF00BF00215C20015500BF019811E705
:105AE000657300088173000873730008E57300088C
:105AF0003D730008704770470249C9690143014A74
:105B0000D16170470000014070B504462546681E0B
:105B10000949884201D901200CE0681E0749486103
:105B20000321081F02F090F9002004498861072032
:105B30000861002070BD0000FFFFFF0000E000E0F2
:105B40000146044A1068044A0A600022014B1A60A8
:105B50007047000094040020E80B002010B50949AC
:105B600009682022114020290AD101684968CAB277
:105B700005490B680968491C034C21600349CA5454
:105B800010BD00000044004094040020E80B0020F9
:105B900010B50446002C01D1012010BDA0690028D9
:105BA00000D000E000BF4D20005D002805D100219D
:105BB0004C200155204600F030F824214D2001559D
:105BC0002068C0680121490388432168C8602046D5
:105BD00001F0AEFF206A002802D0204601F0ECFE62
:105BE000206800690121C902884321680861206892
:105BF000406908218843216848612068C068012104
:105C0000490308432168C8600020206520214D20F9
:105C100001554E2001550020BFE77047FFB583B006
:105C200004460D461746002001904D20005D2028B7
:105C300071D1002D01D0002F02D1012007B0F0BD9D
:105C400001210903A068884208D12069002805D1F4
:105C5000E807C00F002801D00120EFE700BF4C206B
:105C6000005D012801D10220E8E701214C20015507
:105C700000BF0020206521214D200155FEF7B4FE14
:105C800001902786678601210903A068884205D113
:105C90002069002802D10026029502E02E4600204D
:105CA00002901EE006980090002280212046019B71
:105CB00002F010F8002801D00320BFE7002E09D120
:105CC00002980088C005C00D216848600298801CB9
:105CD000029003E0307821684860761C608E401E98
:105CE0006086608E0028DDD1069800900022402159
:105CF0002046019B01F0EEFF002801D003209DE724
:105D000020214D20015500BF00214C20015500BF2E
:105D1000002093E7FFE7022090E700BFFEE70000C6
:105D200001460A48002906D0012906D0022906D0DA
:105D3000032908D105E0064806E0064804E00648C5
:105D400002E0024800E000BF00BF7047801A060072
:105D5000A0860100400D0300E09304007CB50446DA
:105D6000074903C901910090684601F095FA0025A2
:105D70002046FFF7D5FF0546284600F0B9FD7CBD5B
:105D8000C498000801460868406901229202104048
:105D9000800A002815D0D0430A6850610020C862EC
:105DA00020223920425400223A204254C86B042257
:105DB0001043C86300BF00223820425400BF0120B6
:105DC00070470020FCE7F8B505460E461446002053
:105DD00000906A463146284600F0A8FD002807D00A
:105DE0000320FFF7BBFF6A463146284600F09EFDC0
:105DF0006846008820800020F8BD0000FFB581B013
:105E000004460F4615460B9E206800680121890252
:105E100008432168086020680068FF2101310843B9
:105E20002168086000960022484920460A9B00F03D
:105E30003BF9002802D0012005B0F0BDFE2038401B
:105E40002168086133464149491C20460A9A00F0FE
:105E50006DF9002801D00120EEE700BF002000907E
:105E600020684069009020688069009000BF00BFF2
:105E7000324620460A9900F001FA00280BD0E06B68
:105E8000042806D1206800680121490208432168DE
:105E900008600120D0E70498012803D1E8B2216806
:105EA00008611BE0FF200002284000122168086101
:105EB000324620460A9900F0E1F900280BD0E06B49
:105EC000042806D12068006801214902084321689E
:105ED00008600120B0E7E8B2216808613246204638
:105EE0000A9900F0CBF900280BD0E06B042806D10A
:105EF00020680068012149020843216808600120E8
:105F00009AE720680068FF21013108432168086092
:105F1000009600220D4920460A9B00F0C5F8002893
:105F200001D0012088E701203843C0B22168086110
:105F300033460649491C20460A9A00F0F7F8002823
:105F400001D0012078E7002076E700000100010081
:105F5000FFB581B0044615460B9F0A9E2068006875
:105F6000FF2101310843216808603346002234498B
:105F70002046009700F098F8002802D0012005B0D4
:105F8000F0BDFE2102980840216808613B46324678
:105F90002B49491C204600F0C9F8002801D00120F7
:105FA000EDE700BF00200090206840690090206865
:105FB0008069009000BF00BF3A463146204600F09D
:105FC0005DF900280BD0E06B042806D1206800683A
:105FD000012149020843216808600120CFE70498A5
:105FE000012803D1E8B2216808611BE0FF2000020C
:105FF00028400012216808613A463146204600F0E8
:106000003DF900280BD0E06B042806D12068006819
:10601000012149020843216808600120AFE7E8B286
:10602000216808613B46324605497F31204600F031
:106030007DF8002801D00120A1E700209FE70000A3
:106040000100010070B504460D46164623E02046C7
:10605000FFF798FE002801D0012070BD681C0028C1
:1060600019D0FEF7C1FC801BA84201D8002D12D127
:106070000020E06220213920015500213A200155FD
:10608000E06B20210843E06300BF00213820015568
:1060900000BF0120E1E72068406904210840800832
:1060A0000028D4D00020D8E7F8B504460D4617469E
:1060B0001E461DE0701C00281AD0FEF795FC0699BC
:1060C000401AB04201D8002E12D10020E0622021F7
:1060D0003920015500213A200155E06B2021084369
:1060E000E06300BF00213820015500BF0120F8BD4A
:1060F0002802000E01280AD120684069A9B2084090
:10610000A9B2884201D101200BE0002009E02068FB
:106110008069A9B20840A9B2884201D1012000E0FB
:106120000020B842C6D00020E1E70000F8B50446E0
:106130000D4616461F4640E020684069012189024D
:106140000840800A00281BD02068006849100843D6
:10615000216808602748216848610020E06220210A
:106160003920015500213A200155E06B04210843F4
:10617000E06300BF00213820015500BF0120F8BDB9
:10618000701C002819D0FEF72FFCC01BB04201D8AC
:10619000002E12D10020E06220213920015500217B
:1061A0003A200155E06B20210843E06300BF002145
:1061B0003820015500BF0120E1E72802000E012828
:1061C0000AD120684069A9B20840A9B2884201D129
:1061D00001200BE0002009E020688069A9B2084096
:1061E000A9B2884201D1012000E000200028A3D0FC
:1061F0000020C4E7FFFBFFFF70B504460D461646BE
:1062000033E020684069102108400009002812D0BE
:10621000C843216848610020E062202139200155EF
:1062200000213A200155E06BE06300BF38200155A2
:1062300000BF012070BDFEF7D7FB801BA84201D82C
:10624000002D12D10020E0622021392001550021CB
:106250003A200155E06B20210843E06300BF002194
:106260003820015500BF0120E4E720684069402143
:10627000084080090028C4D00020DBE770B5044640
:106280000D46164623E02046FFF77CFD002801D08E
:10629000012070BD681C002819D0FEF7A5FB801BEB
:1062A000A84201D8002D12D10020E062202139201F
:1062B000015500213A200155E06B20210843E0639D
:1062C00000BF00213820015500BF0120E1E7206810
:1062D000406980210840C0090028D4D00020D8E7B8
:1062E000F8B504460D461646002732462946204694
:1062F00000F052FB0746002F13D00320FFF72EFDBE
:1063000032462946204600F047FB08480068401CFA
:106310000649086008460068022805D9FEF794FF80
:1063200002E00020014908600020F8BD6804002058
:10633000FFB5002004240023FD260746401C374DEE
:10634000EE55FC260746401CEE55FB260746401C32
:10635000EE55FA260746401CEE55002901D0A51837
:10636000ACB20546471CB8B22C4F7C55FF252D0218
:1063700025402E120546471CB8B2284F7E55FF26F1
:106380000136009D3543EEB20546471CB8B2234F97
:106390007E55FF260136009D3543FF2636023540E7
:1063A0002E120546471CB8B21C4F7E55039DEEB217
:1063B0000546471CB8B2194F7E55FF263602039D8D
:1063C00035402E120546471CB8B2144F7E550029A1
:1063D00008D0002304E0CD5CC618104FBD555B1CEF
:1063E0009342F8D38518A8B204260546471CB8B2D4
:1063F0000A4F7E5503260546471CB8B2074F7E5507
:1064000002260546471CB8B2044F7E5501260546B4
:10641000471CB8B2014F7E5504B0F0BDF80700200C
:1064200008B500BF1948C06B0121C90208431749CC
:10643000C8630846C06BC9140840009000BF00BF85
:1064400012484030006A0121084310494031086277
:1064500000BF0E484030006A022108400028F8D0F2
:106460000B480C490860032048607D210901094858
:1064700081600949C160FEF74BFE002804D007A0E7
:1064800001F0C4FC00BFFEE708BD000000100240A0
:106490000030004070090020FF0F000048414C5FB1
:1064A000495744475F496E6974204661696C656469
:1064B0000D0A000010B50548FEF756FE002804D06E
:1064C00003A001F0A3FC00BFFEE710BD700900208F
:1064D00048414C5F495744475F526566726573682F
:1064E000204661696C65640D0A00000000B587B044
:1064F00000BF0D48406B012108430B494863084623
:10650000406BC007C00F019000BF00BF0120029088
:106510000390002004900220059002A905200007A6
:10652000FEF782F907B000BD0010024010B500224E
:10653000012105200007FEF751FA10BD10B5012218
:10654000114605200007FEF749FA10BD0148006812
:1065500070470000440200201CB5014600200022C4
:106560000092019200BF31E082008A5E9202C30075
:10657000184CE3589B11D21A009282005218022341
:10658000D35E9A02C3001B195B689B11D21A019259
:10659000C20023469A58009BD218C300E250C200A2
:1065A0002346D2185268019BD218C3001B195A60A7
:1065B000009A921212B28300074CE252019A921290
:1065C00012B283001B195A80421CD0B21028CBDBB8
:1065D0001CBD0000D00D0020900D00207FB50146AD
:1065E00000200022009201920292039200BF59E023
:1065F00082008B5EDA171C0A120622431D06030175
:106600002A4CE41818CCA6059B0A3343A412EB1AB3
:10661000A24100930192820052180223D35EDA173E
:106620001C0A120622431C060301204D5D19AB68AB
:10663000ED68AE059B0A3343AD12E31AAA410293FB
:1066400003920201194B9A1814685268009D019B2D
:1066500064195A410301154DEB181C605A60020180
:106660002B46D2189468D268029D039B64195A4144
:1066700003010E4D5B199C60DA60019A1402009BC5
:106680001A0E224312B28300094CE252039A1402FA
:10669000029B1A0E224312B28300054C1B195A802A
:1066A000421CD0B21028A3DB7FBD0000900E00205A
:1066B000500E00207047000010B50348428803497F
:1066C0000348FFF743F810BD60040020280A0020AB
:1066D0008009002000B501460B0001F0A7FB402116
:1066E00024272A2D3075757575757575757575380E
:1066F000393A3B3C3D3E3F40414243444546474E8C
:106700004F505152535455565758595A5B5C5D5F20
:10671000606162636465666768696A6B6C6D6E75FB
:106720002A48007900BD29484079FBE7274880794D
:10673000F8E72648C079F5E724488068F2E724485E
:106740000088020423480078401C1018EAE700BFC4
:1067500000BF00BF00BF00BF00BF00BF00BF00BF41
:1067600000BF00BF00BF00BF00BF00BF0846103819
:10677000820016480C308058D4E700BF00BF00BF2D
:1067800000BF00BF00BF00BF00BF00BF00BF00BF11
:1067900000BF00BF00BF00BF0020C3E700BF00BFB5
:1067A00000BF00BF00BF00BF00BF00BF00BF00BFF1
:1067B00000BF00BF00BF00BF00BF084630388200E6
:1067C00002484C308058ADE70348ABE7C4030020D3
:1067D000AE040020AC040020FFFFFF7F70B505462B
:1067E0000C462B0001F022FB402124272A2D77772D
:1067F00077777777777777777735363738393A3BE2
:106800003C3D3E3F40414243444B4C4D4E4F505126
:1068100052535455565758595A61626364656667B6
:1068200068696A6B6C6D6E6F707730490C7155E0FA
:106830002E494C7152E02D498C714FE02B49CC719F
:106840004CE0002C01DD204600E001202749886053
:1068500044E000BF00BF00BF00BF00BF00BF00BFDB
:1068600000BF00BF00BF00BF00BF00BF00BF00BF30
:106870002846103881001D480C3044502EE000BFDF
:1068800000BF00BF00BF00BF00BF00BF00BF00BF10
:1068900000BF00BF00BF00BF00BF00BF28462038B8
:1068A000810012484C30445018E000BF00BF00BFC8
:1068B00000BF00BF00BF00BF00BF00BF00BF00BFE0
:1068C00000BF00BF00BF00BF284630388100074826
:1068D0004C30445002E00020C04370BD00BF3F2D4B
:1068E00001D1FCF755FD0020F7E70000C4030020AC
:1068F00010B504460A480B49086008464460002168
:106900008160C160016141618161C161FEF778F818
:10691000002804D004480068401C0349086010BDEA
:10692000005400402009002068040020F0B585B024
:1069300004460D46164600200490032003900027CD
:1069400012E06420022104AA012300920191029026
:106950002A4621460F48FEF72DF90746002F00D1A1
:1069600008E00120FDF7F2FD0398411EC9B2039132
:106970000028E6D100BF6946088A0006000C098A93
:10698000FF2212021140091208433080384605B038
:10699000F0BD00002009002037B584B004460D4644
:1069A0006846008B0006010C6846008BFF2212022D
:1069B00010400012014306916420022106AA01231F
:1069C0000092019102902A4621460248FEF78AFA77
:1069D00007B030BD2009002000487047C4030020E4
:1069E0008C207047704710B5FEF7D2FB00F072FFA5
:1069F0000320FFF7B3F900F023FC01F03DF800F0AD
:106A000053FC01F0B5F9FFF771FDFFF78FFDFFF7BC
:106A100007FD10BD0A480068002810D0094800682A
:106A2000401C0849086008460068FF21433188423D
:106A300005D9012004490860002001490860704719
:106A4000500400205404002058040020F0B587B002
:106A500000200690FE48007800287DD0FD48007890
:106A6000AA287AD1FFF726FDFA488078F821084055
:106A7000C010F9490880F74840780007C00D098820
:106A80004018F5490880F5480078002817DDF348DC
:106A90000078401EF1490870EF48008807280AD1A5
:106AA000EF48FDF7C1FB0121ED48FDF74AFBEC483B
:106AB000FDF770FA04900020E74908807DE2E54880
:106AC000FCF72AF8E7480078002806DDE24802884B
:106AD000E5490020FBF73CFF6FE2E448007801281D
:106AE00011D1E048007800280DD1DB480088072844
:106AF000E4D101F02FFC0020DD490870DD49087069
:106B0000DA49087059E2DB480078002875D0D5488A
:106B10000078002871D1D548007800286DD1D5487B
:106B2000007801282FD1D2480078012816D1CA4810
:106B300000880728C2D101F0C9FF0220CD490870A2
:106B4000CD484088C849CD4B0022009101901146A4
:106B5000012001F02DFE30E240E226E2BE4800882E
:106B60003F28ABD101F0B2FF0220C2490870C248F1
:106B70004088BD49C14B002200910190114601207F
:106B800001F016FE19E2BB480078022807D1B2488E
:106B900000883F2892D10320B64908700DE2B5481D
:106BA000007803288AD1AC4800883F280BDAB24825
:106BB0004088AD49B14B002200910190012110465F
:106BC00001F0F6FDF9E1A44800883F2884D1AA48E5
:106BD0004088A549A94B012200910190114600204F
:106BE00001F0E6FDA548007801288BD1A349087083
:106BF0000020A0490870E0E1FFE7FFF7A7FC0028AC
:106C00007ED09F480078012835D1934800883F28DE
:106C100031D100209A490870002409E00020A10029
:106C2000984A5050A100984A505098490870641CE6
:106C3000102CF3DBFD2096490870FC204870FB20E7
:106C40008870FA20C870042008710020487109205B
:106C500088710120C871002008724872042088726F
:106C60000320C87202200873012048730E2188484F
:106C700002F0CEFB43E08248007802283FD17648FC
:106C800000883F283BD100207D490870814800885A
:106C900069210902884201DD00270CE07D4909884D
:106CA00069221202511A64225143084669210902DD
:106CB000FBF734FAC7B2FD2075490870FC20487014
:106CC000FB208870FA20C8700620087100204871E7
:106CD0000A2088710120C871002008724872084695
:106CE00087720020C87204200873032048730220B2
:106CF00088730120C8731021654802F089FB00E009
:106D0000F1E06448008869210902884205DD614894
:106D10000088401E5F4908804FE15E4800880128D6
:106D200024DD5C480088401E5A4908805A4805AB5B
:106D30000090494802884C49002002F013F9464867
:106D400000883F28E8D1FBF7C9FD80215348FBF7B5
:106D500012FA40215248FBF70EFA40215148FBF746
:106D60000AFA80215048FBF706FA26E149480088D4
:106D70000128D1D1384800883F28CDD14548008826
:106D8000401E44490880FFF727FE0546002444E0E2
:106D900046480078FBF7EAFAA1003A4A01905058B9
:106DA000FBF7E4FA00900199FBF75AFA4049029088
:106DB000FBF793FA0390FBF7E0FA0646C82E05D2DC
:106DC000C821A20028460C30815003E0A1002846CB
:106DD0000C30465037480078FBF7C8FAA1002A4A21
:106DE00001905058FBF7C2FA00900199FBF738FA6E
:106DF0002F490290FBF771FA0390FBF7BEFA0646A3
:106E0000C82E05D2C821A20028464C30815003E08C
:106E1000A10028464C304650641C102CB8DB0020E2
:106E200025490880022410E0A10028460C30405873
:106E3000A100224A5158884206D90120A0401E498B
:106E4000098840181C490880641C102CECDB37E0D2
:106E50006C040020280A0020CE000020CB00002077
:106E6000840B0020CA000020E4050020C700002099
:106E7000C9000020C800002060040020CC000020D1
:106E8000C60000201C0500205C050020C00000207A
:106E90009C050020C2000020DC0000209010002093
:106EA00050100020900F0020D00F0020C4000020C0
:106EB00000002041C5000020DE0000208095000871
:106EC000FCF766FA80214A48FBF755F9402149480A
:106ED000FBF751F940214848FBF74DF9802147481D
:106EE000FBF749F969E0464800883F2805D1454845
:106EF0000078002801D100F0B3F8434805AB0090BA
:106F00003F4802884149002001F02AFE3C480088A1
:106F10003F2852D13E4800883E4908806846808A12
:106F20003B4908803B4909884800C10F0918C9033B
:106F3000090C384A1180FFF709FB002824D100F022
:106F4000E7FC04280FD16846818A2F48007800F0BA
:106F50005DFC2D480078002802D1FFF7E7FA13E026
:106F6000FFF7ECFA10E028480078002805D12AA0A5
:106F700000F04CFFFFF7DAFA06E02648018828A067
:106F800000F044FFFFF7DAFA80211948FBF7F3F825
:106F900040211848FBF7EFF840211748FBF7EBF8C2
:106FA00080211648FBF7E7F807E000201449088025
:106FB0000D20FCF781FBFCF761FB00201C490870E9
:106FC000FFF77AFB0E4800883F2802D10120069087
:106FD00001E000200690069807B0F0BD094800784F
:106FE000002801D100F042F9002006900698F3E74E
:106FF0009010002050100020900F0020D00F002093
:10700000CE00002041020020DC000020E40500202A
:10701000D8000020DA0000204F46460D0A0000008C
:1070200064697374616E63653A25640D0A0000003B
:107030006C04002010B500240AE0A000074BC01823
:107040004288A000195C402002F0C6F8601C84B29F
:10705000A0000249085A0028EFD110BD9A980008F4
:1070600010B500240AE0A000084BC0184288A00018
:10707000195C402002F0B0F8601C84B2A000034903
:10708000085A0028EFD100F0B5FB10BD7698000833
:1070900038B50024002100916A460121402002F009
:1070A0008DF868460088012109030840002801D0B6
:1070B000012418E06846008804210840002801D017
:1070C000002410E06846008810210840002801D004
:1070D000022408E06846008802210840002801D008
:1070E000032400E00424204638BD08B500210091A7
:1070F0006A460421402002F061F868460088C00614
:10710000400E08BD08B5402100916A460521402087
:1071100002F054F86846008808BD08B500210091C7
:107120006A464421402002F049F86846008808BDBC
:1071300038B5FF210131009100246A460421402026
:1071400002F03CF8684600884005440F052C03DA3D
:1071500060000249085A38BD4020FCE76C980008DE
:1071600010B5002400F0C2F80A20FCF7A5FA23E0CD
:10717000A0003249085A6D2802D1601C84B21BE07D
:10718000A0002E49085A702802D1601C84B213E076
:10719000A0002A49085A722802D1142C00DD10E000
:1071A000A000264BC0184288A000195C402002F0C5
:1071B00013F8601C84B200BFA0002049085A0028C0
:1071C000D6D100BF0AE0A0001C4BC0184288A00026
:1071D000195C402002F000F8601C84B2A00017493E
:1071E000085A0028EFD1FCF72DFA00241DE0A0007A
:1071F0001249085A6D2808D1A0000B46C0184288D1
:10720000A000195C402001F0E7FFA0000B49085ADC
:10721000702808D1A0000B46C0184288A000195C55
:10722000402001F0D9FF601C84B2A0000349085A35
:107230000028DCD100F064F810BD00002897000899
:1072400010B500240AE0A000074BC0184288A00037
:10725000195C402001F0C0FF601C84B2A00002490C
:10726000085A0028EFD110BD0497000810B5064851
:107270000068012806D1FFF7DDFEFFF71DFA0020A8
:107280000149086010BD0000580400200149086051
:10729000704700003C020020024A416851600168CA
:1072A00011607047BC03002000B587B000BF0D48D7
:1072B000406B022108430B4948630846406B02219A
:1072C0000840019000BF00BF2020029001200390E1
:1072D000002004900220059002A90348FDF7A4FABB
:1072E00007B000BD001002400004005010B500229D
:1072F00020210248FDF772FB10BD00000004005081
:1073000010B5012220210248FDF768FB10BD0000E6
:107310000004005010B50248FDF7F2FF10BD000058
:107320008009002070B505466C6A00214620015393
:107330000020E0872046FDF7CFFF70BD70B5054601
:107340006C6A206840688008800021684860206E70
:1073500010210843206601215D2001552046FDF7DC
:10736000BBFF70BD70B50446656A2846FEF7BAFAE1
:1073700070BD70B50446656A2846FEF7BCFB70BD5B
:1073800070B505466C6AFDF72FFB06462868006855
:1073900020210840202820D02068406888432168A8
:1073A0004860206840688008800021684860324654
:1073B0006421204600F054F8002801D020202066E7
:1073C00000214620015301215D200155206E002837
:1073D00003D02046FDF780FF70BD2046FEF778FA07
:1073E00000BFF9E770B505466C6AFDF7FDFA064681
:1073F0002868006820210840202824D020684068A0
:1074000088432168486032466421204600F06FF8C6
:10741000002803D0206E20210843206620684068A1
:1074200080088000216848600020E0870021462015
:10743000015301215D200155206E002803D0204614
:10744000FDF74AFF70BD2046FEF754FB00BFF9E789
:1074500010B50248FDF722FF10BD00008009002092
:10746000F8B504460E461546FF210531606888428E
:107470000ED10121C903A068884203D04911A06838
:10748000884205D12068006840218843216808604F
:107490003346002280212046009500F0D3F80028D2
:1074A00005D0206E2021084320660320F8BDFF216F
:1074B00005316068884218D10121C903A06888425B
:1074C00003D04911A06888420FD13346002203211E
:1074D00049022046009500F071F8002805D0206E82
:1074E0002021084320660320E0E70020DEE7F8B50E
:1074F00004460E461546334600220321C9022046A3
:10750000009500F05BF8002805D0206E202108438C
:1075100020660320F8BD33460022802120460095D6
:1075200000F090F8002805D0206E20210843206646
:107530000320EFE73346002203214902204600954D
:1075400000F03CF8002805D0206E2021084320667A
:107550000320DFE70020DDE710B504461448154995
:10756000086008211348C161002181604161016107
:1075700081620721C1620902C1600021016281614B
:10758000416241630121016300200A4948600846C5
:10759000FDF76CFF002801D000BFFEE7012040028C
:1075A000FEF7AAFA224604490248FEF7CFF810BDBA
:1075B0000030014080090020280A0020F8B5044668
:1075C0000E4617461D4636E003204002864203D190
:1075D000002F01D12068007B681C00282BD0FDF70C
:1075E00003FA0699401AA84201D2002D23D120683F
:1075F0004068E021884321684860FF2105316068C8
:1076000088420ED10121C903A068884203D04911E4
:10761000A068884205D1206800684021884321681D
:10762000086001215D20015500BF00215C2001554B
:1076300000BF0320F8BD206880683040B842C3D145
:107640000020F7E7F8B504460E4617461D462EE023
:10765000681C00282BD0FDF7C7F90699401AA842EC
:1076600001D2002D23D120684068E02188432168A1
:107670004860FF210531606888420ED10121C903AD
:10768000A068884203D04911A068884205D12068CB
:107690000068402188432168086001215D20015570
:1076A00000BF00215C20015500BF0320F8BD206809
:1076B00080683040B04201D1012000E00020B84293
:1076C000C6D10020F2E7704710B5454A1278454B05
:1076D0001A80434A92785A801A461288FF2A03D0A9
:1076E0001A465288FF2A04D11E223E4B1A800322DA
:1076F0005A803C4A12881E2A03DC3A4A5288032ADE
:1077000004DD1E22374B1A8003225A80354A128824
:10771000D200354BD2185288324B9A801A461288C2
:107720005200521C9200304BD21852882D4BDA80F6
:107730001A4652889300D21892002C4BD2185288C5
:10774000284B1A811A4652889300D218521C920074
:10775000264BD2185288234B5A811A4652889300DE
:10776000D218921C9200214BD21852881D4B9A813C
:107770001A4652889300D218D21C92001B4BD21882
:107780005288184BDA811A4652889300D218121D7B
:107790009200164BD2185288124B1A82002009E030
:1077A00042000F4BD2189188114A914200D103E058
:1077B000421CD0B20728F3DB00BF0D4A91420DD026
:1077C000002009E04200064BD2189388821C520028
:1077D000044CA352421CD0B20728F3DB10BD0000BA
:1077E00000BB000890070020E6000020DE0100201A
:1077F000FFFF0000012003490860002002490860E3
:10780000704700005004002054040020F0B5A1B0DF
:1078100006460D46832023490870002048703746ED
:1078200021480078052803D120480078012802D09B
:1078300038461030C7B21B4887700146CD70280407
:10784000000E0871002406E0A00019490858A100A4
:1078500001AA5050641C102CF6DB102408E02046CE
:107860001038800013490858A10001AA5050641C28
:10787000202CF4DB002405E001A8015D0948401D2F
:107880000155641C802CF7DB04210B4801F0C0FD7E
:107890008521044801F0BCFD0421084801F0B8FD31
:1078A00021B0F0BD9C050020A0040020A104002010
:1078B000900F002050100020789500087C9500085B
:1078C00010B5FDF759FCFFF7A5F800F017F9FEF722
:1078D000F1FD10BD014802490860704700366E0195
:1078E0008404002007484068000C00040121C903FB
:1078F000401805490969084302494860C80303491B
:107900008860704700100240000FFF1F00ED00E08C
:107910000148008880B2704742020020004870474A
:107920006C07002070B504460D46002C01D0002DD8
:1079300000D170BD20B2054948802246294603483F
:10794000001DFAF7FFFB00BFF3E700006C07002003
:10795000F0B585B005460E4614461F46002004903B
:107960000390A54200DB2546A64200DB26466100C7
:10797000491B891B4800FAF7EEFC0290701BFAF7CE
:10798000EAFC01900299FAF7A8FC04903846FAF74D
:10799000EDFC00900499FAF70AFC06490190FAF709
:1079A0005FFC0290FAF7E9FC80B20390039805B0FF
:1079B000F0BD000000008C424022016A1140002905
:1079C00015D00168496992019143426A11430268E6
:1079D000516101221203416A914208D1016849694B
:1079E000032252039143826A114302685161704736
:1079F00000B587B000BF1F48406B012108431D49F7
:107A000048630846406BC007C00F019000BF00BF2D
:107A100000BF0846C06B0121490408431549C863EB
:107A20000846C06B012149040840019000BF00BF17
:107A3000042002900220039001200490022005906F
:107A40000420069002A905200007FCF7EDFE0220A5
:107A500002900920069002A905200007FCF7E4FE29
:107A6000012200211C20FDF7E5FB1C20FDF7D0FBC7
:107A700007B000BD0010024010B5FFF7B9FF1D4868
:107A80001D490860E1204002486000211A488160D9
:107A9000C1600161816108214161FEF779F81548F3
:107AA00015490860E12040024860002112488160C9
:107AB000C160016181610C214161FEF769F80E48E6
:107AC0000068C068FF21013108430B490968C8609C
:107AD000094800684069012108430749096848616D
:107AE00005480068C0682021084303490968C86048
:107AF00010BD000000440040300B00200948006821
:107B000000280ED008480068401C07490860084655
:107B100000680A2805D901200449086000200149AD
:107B20000860704770040020740400208004002066
:107B3000FEB5044620680069012149038843E168D5
:107B40000843216808612169A06808436169084306
:107B500002902068C0685E49084002990843216885
:107B6000C860E0690290206840690121C902884329
:107B7000029908432168486120684069032109028D
:107B80008843A1690843216848610121C902E0696D
:107B900088424ED1FDF76EFB0546626851001922FE
:107BA0006A431046FAF7A4FA06466421FAF7A0FAE7
:107BB00007016268510019226A431046FAF798FAE1
:107BC00006466268510019226A431046FAF790FA95
:107BD00064210090FAF78CFA64214843301AC000FF
:107BE00032300190FAF784FAF821084040003F183B
:107BF0006268510019226A431046FAF779FA06467C
:107C00006268510019226A431046FAF771FA64213A
:107C10000090FAF76DFA64214843301AC000323000
:107C20000190FAF765FA4007400F3818216888601C
:107C30004CE0FDF71FFB05466268910019226A437C
:107C40001046FAF755FA06466421FAF751FA070189
:107C50006268910019226A431046FAF749FA06460B
:107C60006268910019226A431046FAF741FA6421CA
:107C70000090FAF73DFA64214843301A000132308F
:107C80000190FAF735FAF02108403F186268910038
:107C900019226A431046FAF72BFA064662689100E9
:107CA00019226A431046FAF723FA64210090FAF782
:107CB0001FFA64214843301A000132300190FAF76C
:107CC00017FA0007000F381821688860FEBD000011
:107CD000F3E9FFFFFFB581B004460D4617460A9E43
:107CE00024E0701C002821D0002E05D0FCF77CFE7B
:107CF0000499401AB04219D92068C068FF21A13107
:107D000088432168C86020684069400840002168B5
:107D1000486120214D2001554E20015500BF002112
:107D20004C20015500BF032005B0F0BD206800685D
:107D30002840A84201D1012000E00020B842D0D064
:107D40000020F1E710B500F001F810BD10B50548AE
:107D5000FDF704FF00200449086001200349086082
:107D600010BD0000300B00207404002070040020BF
:107D700000B587B000BF0E48406B012108430C4995
:107D800048630846406BC007C00F019000BF00BFAA
:107D900008480290032003900020049002200590E0
:107DA00002A905200007FCF73FFD07B000BD000059
:107DB000001002400810000010B5FFF769F91249E1
:107DC0000880FFF79FF910498880FFF7A6F90E4950
:107DD000C880FFF7ADF90C494880084600880028A4
:107DE00004D1084680888000083003E006484088B7
:107DF000800008300449088108460088022801D123
:107E00007420088110BD0000060900200FB410B5D1
:107E100003A9044B044A029800F062F810BC08BCA5
:107E200004B01847298400081805002030B47446AF
:107E3000641E2578641CAB4204D3635D5B00E318C9
:107E400030BC18471D46F8E710B5002819DB1A4A60
:107E500003231B02D21883089B00D2588307DC0E31
:107E6000FF23A3409A438B071B0E8407E40EA34015
:107E70001A43114B032424021B198408A4001A512D
:107E800018E00E4A03071B0F083B9B089B00D258C3
:107E90008307DC0EFF23A3409A438B071B0E840746
:107EA000E40EA3401A43054B0407240F083CA40822
:107EB000A4001A5110BD000000E100E01CED00E03C
:107EC00002E008C8121F08C1002AFAD170477047A3
:107ED000002001E001C1121F002AFBD17047000001
:107EE000FFB58DB00446002506E025280AD0109A7B
:107EF0000F999047641C6D1C20780028F5D1284606
:107F000011B0F0BD00270121484A009700E0074367
:107F1000641C23780846203B98401042F7D1207813
:107F20002E2817D1042007436078641C2A280CD11E
:107F30000E98641C02C800910E900BE000990A2272
:107F4000514330394018641C009020780146303984
:107F50000929F3D920780028D1D0642808D06928CD
:107F600006D075281ED0109A0F9990476D1C5BE0C3
:107F70000A200E99019001C90E91002802DA4042B0
:107F80002D2102E0390504D52B216A461172012109
:107F900003E0F90704D02021F7E70BAE0B910DE0C9
:107FA0000021FAE70A200E99019001C90E91F7E726
:107FB0000199FAF79DF83031761E31700028F7D11B
:107FC00003A8801B20300190780701D5009801E0BC
:107FD000012000900199884201DD401A00E0002054
:107FE0000027009006E002A8109AC05D0F99904704
:107FF0006D1C7F1C0B988742F5DB04E0109A302043
:108000000F9990476D1C0099481E00900029F5DCDF
:1080100005E03078109A761C0F9990476D1C0199F5
:10802000481E01900029F4DC641C65E70928010062
:1080300001460020002901DB0A4601E00122521A14
:1080400090B2704701460020002901DB0A4601E09A
:108050000122521A10467047FCB502460B46002119
:10806000002422E08C4210DAE500AE1860CE0196C2
:108070000095E500AD18CE00B618C0CEC0C5CD0045
:10808000AD18019F009EC0C500BF1D46DE0F7619CA
:10809000701004E0091A0546C60F76197010814267
:1080A00001DB0028F6DC0918641C9C42DADBFCBD0D
:1080B00010B5FF22453202490248FAF743F810BDD5
:1080C0002C990008380C002010B51F4B1988CB17CD
:1080D0009B0F5B189A1081001C4B5B5884001C4955
:1080E00009595B1A84001A4910390959591A830031
:1080F000174C203CE358C91A1301164C1B19840075
:1081000019518100114B5B588400114909595B1AC0
:1081100084000F4910390959591A83000C4C203C2E
:10812000E1508100094B5B588400094909595B1AE9
:108130008400074910390B518100044B5B588400BF
:1081400003490B5110BD0000C40400201011002091
:108150006011002070110020F3B589B00A990998C8
:10816000FFF77AFF022495E021462020F9F7D6FF99
:108170000890002689E0002580E0089969430846B8
:10818000C917090F091809110901411A8900444A40
:1081900051580791089969430846C917090F0918EA
:1081A00009110901411A89003E4A51580691701976
:1081B000C1000998091803C905910490E10F091934
:1081C000491072198918CA000094099988580799AA
:1081D00000F020F90746E10F0919491072198918B2
:1081E000CA000194099951184868069900F012F9DB
:1081F000381A0290E10F0919491072198918CA003A
:10820000009409998858069900F004F90746E10F8F
:108210000919491072198918CA000194099951184D
:108220004868079900F0F6F8381803900299049806
:1082300041187019C2000998815003990598411896
:108240007019C200099810184160029A0499891A9D
:108250002046E20F121852107319D218D300099A4F
:10826000D150039A0599891AE20F12185210731906
:10827000D218D300099A9A1851606D1CE10F0919A0
:108280004910A94200DD78E736190A98864200DADB
:1082900071E764000A98844200DC65E70BB0F0BD2A
:1082A000EC9A00082C9B0008F8B50546002417E05E
:1082B00020011B494018A9004058E100194A5050BC
:1082C000E000114608586100174A515A484380128D
:1082D000E100144A50500020E10089184860641CF5
:1082E000202CE5DB20210F48FFF736FF002414E0A7
:1082F000E1000C4A5058FFF7A5FE0646E100094A86
:1083000089184868FFF79EFE074639463046FBF756
:1083100087FAE100034A5050641C202CE8DBF8BDCA
:108320007011002070130020D804002030B50346DF
:108330000C46FF20092106E08D005D5B954201D1CE
:10834000C8B204E0491C2546093D8D42F4DC00BF5B
:1083500030BD000010B5FF22453226492648F9F706
:10836000F1FE264881882448A83041802348C188EE
:108370002148AC304180214801891F488C30418020
:108380001E4841891C48903041801C4881891A4808
:10839000943041801948C189174898304180174866
:1083A000018A15489C30418002219C384183144940
:1083B000C1830121C187134940304180FF216F31C2
:1083C000143041801B214902001D41800E495C3060
:1083D000418083218900001D41800C49001D41809E
:1083E00021214902001D418009497430418000F07B
:1083F00001FF10BD2C990008380C002090070020C8
:10840000E02200003844000019100000016900005B
:10841000248E00000246104648430346C017800DD4
:10842000C01880127047000013B50C46034B0122A0
:1084300069460348FDF7F2FB00981CBDFFFF0000F2
:10844000300B0020F8B50746002600BF012F10D1E1
:1084500000204A49088030214948F9F78CFE302134
:108460004848F9F788FE79024748F9F784FE304614
:10847000F8BD00F021FE002403E0204600F08AF859
:10848000641C042CF9DB3D490888C117890F0918C1
:1084900089108900411A032907D1002403E02046EE
:1084A000FFF712FE641C042CF9DB344800887F2897
:1084B0001EDB002419E02046FFF7F6FE02250DE042
:1084C000E80032490858A100314A51588A01511A2E
:1084D000884202D9201DC6B202E06D1C0F2DEFDBD1
:1084E00000BF002E00DD02E0641C042CE3DB22E070
:1084F000224800881F281ED1002419E02046FFF7DB
:10850000D3FE04250DE0E80020490858A100204AC8
:1085100051588A01511A884202D9201DC6B202E080
:108520006D1C0F2DEFDB00BF002E00DD02E0641C90
:10853000042CE3DB00BF114800887F280BDB002000
:108540000E49088030210E48F9F715FE30210D48FC
:10855000F9F711FE0FE0094800881F2805D10748E8
:108560000088401C0549088005E004480088401C3C
:1085700002490880FF2630467AE70000C404002044
:1085800010110020401100207011002070130020F5
:10859000C804002010B5021D9200184B9A58184BC1
:1085A0009A4201D9194604E0021D9200134B9A5ACF
:1085B00091B28300134AD25853188400114A103ADA
:1085C00012599A1883000F4C203CE358D2188300AC
:1085D000E25083000B4AD25853188400094A103ADB
:1085E00012599B188400074A103A13518300103225
:1085F000D25853188400034A135110BD5010002064
:10860000FFFF000030110020FFB582B00746484848
:1086100000780830C01B84B2454840780830039980
:10862000401A85B2102C01DD41480478102D01DD7F
:108630003F48457860014019694608803C48807889
:1086400008300499401A84B23948C0780830059936
:10865000401A85B2102C01DD35488478102D01DDDB
:108660003348C57860014019694648803048007831
:108670000838C01984B22E48407808380399401849
:1086800085B2102C01DD2A480478102D01DD284820
:108690004578600140196946888025488078083807
:1086A0000499401884B22248C078083805994018C7
:1086B00085B2102C01DD1E488478102D01DD1C4888
:1086C000C5786001401981B26846C180612251219C
:1086D0001848FFF72BFE064668460088B100154A89
:1086E00089184880622251211248FFF71FFE064672
:1086F00068464088B1000F4A89184880632251219A
:108700000C48FFF713FE064668468088B100094A08
:1087100089184880642251210648FFF707FE064663
:108720006846C088B100034A8918488006B0F0BD89
:10873000A3040020380C002010B5002400BF1BE06B
:10874000A0001049085A61280BD0A000085A6228DE
:1087500007D0A000085A632803D0A000085A642854
:1087600008D1A000074BC0184288A000195C402027
:1087700000F032FD601C84B2A0000249085A0028B3
:10878000DED110BD380C002010B510210648F9F7D5
:10879000F2FC002404E005486100034A5052641CC6
:1087A000042CF8DB10BD0000280C0020FF7F000027
:1087B000FFB585B0074615461E46002400200490EC
:1087C00003900290012F08D1A6480078002803D119
:1087D0000120A449087000E00027012F09D0069865
:1087E000012806D09F480078002801D1002400E02D
:1087F00007240027012D02D104209A4908709948C6
:1088000000780300FFF712FB0504050A2425C400C5
:10881000BFE000F035FD01200390BAE00F990E98FB
:1088200000F040FD9048007810280EDA8E4800785D
:10883000401C8D490870084603780278017800785A
:10884000FFF7E2FEFFF778FF01E001200290A0E0D1
:108850009FE000F0FFFC0490049800283FD183487B
:108860000078401C0D2810DB81480078401C03284C
:108870000BDB00BF0220F9F73BFE05E06420FAF7AE
:108880001BFF7CA0FFF7C2FAF8E77949774800F0B0
:1088900051FD00280BD000BF0220F9F729FE05E0AA
:1088A0006420FAF709FF73A0FFF7B0FAF8E7FF2298
:1088B00045327B497B48F9F745FC00206A4908703E
:1088C000FFF762FF68480378027801780078FFF7C5
:1088D0009BFE00F047FD00F08DFC0A2457E0FF22CC
:1088E00045326F496F48F9F72DFC6F48C37A427AD9
:1088F000817A007A0190FFF787FE00F033FD0221B4
:10890000684841836949C1830121C1876849403072
:108910004180FF215031143041806649001D418063
:1089200065495C30418083218900001D4180634995
:10893000001D418021214902001D418060497430A1
:10894000418000F057FC0120F9F7D2FD5548A830CE
:1089500040885C4988805348AC304088C880514882
:108960008C30408808814F489030408848814D487D
:108970009430408888814B4898304088C881494865
:108980009C304088088201204F490870082400E08C
:1089900000BF00BF334800780300FFF747FA050423
:1089A00008132731430000202E4948703BE003980C
:1089B000012803D102202B49487002E000202949F8
:1089C000487030E00298002803D102202549487001
:1089D0000BE00298012805D1012D03D10420214983
:1089E000487002E003201F4948701CE0012D03D1AC
:1089F00004201C49487002E003201A49487012E024
:108A0000092C03D10020174948700AE00A2C03D131
:108A100002201449487004E0082C02D100201149BA
:108A2000487000E000BF00BF0E4840780D49087054
:108A300008460078002803D1002C01D130700EE0E8
:108A400008480078002804D1002C02D001203070A2
:108A500005E004480078002801D00220307009B0F9
:108A6000F0BD00009A040020A2040020A004002011
:108A7000A10400204C4F505F4641494C2D2D2D2D17
:108A80002D2D2D506F776572206F6E2061676169A3
:108A90006E2D2D2D2D2D2D2D2D2D2D2D0A0000006F
:108AA0002C990008380C0020280C0020E02200003F
:108AB0003844000080B10000191000000169000076
:108AC000248E000090070020410200200020014970
:108AD000087070479A040020002408E0A0001449A0
:108AE00040180068A100134A5050601CC4B2302CDA
:108AF000F4DB0120400710498860FDF774FFF9F7A7
:108B000083FEFAF70FFCFEF72BFBFAF7F3F80020D1
:108B10000A490870FDF7D0FD09E00025FDF796FF32
:108B20000546002D03D0FAF7EDF8FAF79BFCF4E7C1
:108B3000002000080000002000ED00E06C04002090
:108B400070B505460C46224629460348F9F7FAFA5D
:108B50000248046070BD000004070020E00000200F
:108B6000FFB587B015460898FDF7F6FC0898FDF7A5
:108B700035FD00248CE02846E917890F0918891073
:108B80008900691A06D10020E100E94A5050E1004D
:108B9000891848602846E917090F091809110901C1
:108BA000691A06D10020E100E24A5050E10089181C
:108BB0004860E000DE490858A100DF4A515E4018D5
:108BC000E100DB4A5050E000114640184068A10027
:108BD000D94A891802228A5E8018E100D44A89188D
:108BE0004860E000D3490858A100D44A515E4018BB
:108BF000E100D04A5050E000114640184068A10002
:108C0000CE4A891802228A5E8018E100C94A891872
:108C100048602846E917890F091889108900691AE0
:108C2000032915D1E100C24A89184868FFF70AFAFA
:108C3000E100BF4A02905058FFF704FA01900299F0
:108C4000FAF7EEFDA100BE4A51584018A10050505D
:108C50002846E917090F091809110901691A0F298E
:108C600015D1E100B34A89184868FFF7EBF9E10034
:108C7000B04A02905058FFF7E5F901900299FAF7CF
:108C8000CFFDA100AF4A51584018A1005050641CBC
:108C9000102C00DA6FE73F2D77D1FDF79DFE029093
:108CA00000200490069001242AE0A7480079E10002
:108CB000091B884206DAA4484079C01DE100091B5F
:108CC000884206DCA0484079072801DC012C00D04E
:108CD00015E0A0009A490958A2009B480C30805822
:108CE00081420BD9A000964909580698814205D9BE
:108CF000A000934908580690E0B2049000BF641C9D
:108D0000102CD2DB002005900698002819D004987A
:108D1000401C80008A49085801900498401E800039
:108D200008580090049B069A0199FEF711FE0590E1
:108D3000854841790A2041430598814201DC0020A1
:108D4000059082480078002806DD002005907F48C5
:108D50000078401E7D490870002004900690012490
:108D60002BE079480079E100091B884206DA764851
:108D70004079C01DE100091B884207DC7248407938
:108D8000072801DC012C01D016E0CEE0A0006D49DF
:108D90000958A2006C484C30805881420BD9A00081
:108DA000684909580698814205D9A00065490858C4
:108DB0000690E0B2049000BF641C102CD1DB0027A9
:108DC0000698002817D00498401C80005D49085878
:108DD00001900498401E800008580090049B069A59
:108DE0000199FEF7B5FD0746574841790A204143EE
:108DF000B94200DC002700260598002813D1002F77
:108E000011D153480078012808DB0020FFF71AFB36
:108E10000646002E0ED14F4908700BE00120FFF7E7
:108E200011FB064606E00120FFF70CFB064600207A
:108E300048490870002E26D0FF2E24D042480079E1
:108E4000F100891B884205DA3F484079F100891B0F
:108E5000884200DC00263046F9F788FA3E49009047
:108E6000F9F7FEF90190F9F788FA87B236484079A8
:108E70000A214843B84204DC002700260020354977
:108E80000870344806703548007800280DDD00274A
:108E900032480078401E314908700846007828287A
:108EA00003D108460078401F0870324639460598BD
:108EB000FAF7BEFE03900398012802D128490870F2
:108EC0000EE00398002804D1254908702149087054
:108ED00006E00398022803D1214800782049087051
:108EE0001F480078012802D11949087005E01C4884
:108EF0000078002801D1164908701648007800282B
:108F000006DD13480078012802D1022010490870BC
:108F10000F480178109801700D480278394605987D
:108F2000F9F764FD0A99088000BF0BB0F0BD00009E
:108F3000D00F002090100020900D0020500E002037
:108F4000900F002050100020C4030020B304002024
:108F5000D6000020B204002000008C42B40400209F
:108F6000B1040020FEB50E461546089F3046FDF7B9
:108F7000F3FA3046FDF732FB00248CE02846E9176F
:108F8000890F091889108900691A06D10020E100AB
:108F9000434A5050E100891848602846E917090FF4
:108FA000091809110901691A06D10020E1003D4A9A
:108FB0005050E10089184860E00039490858A10084
:108FC000394A515E4018E100354A5050E0001146E0
:108FD00040184068A100344A891802228A5E80182D
:108FE000E1002F4A89184860E0002E490858A10086
:108FF0002E4A515E4018E1002A4A5050E0001146C6
:1090000040184068A100294A891802228A5E801807
:10901000E100244A891848602846E917890F091891
:1090200089108900691A032915D1E1001C4A8918A1
:109030004868FFF707F8E100194A01905058FFF718
:1090400001F800900199FAF7EBFBA100184A51587A
:109050004018A10050502846E917090F09180911B6
:109060000901691A0F2915D1E1000E4A89184868CB
:10907000FEF7E8FFE1000B4A01905058FEF7E2FFCF
:1090800000900199FAF7CCFBA1000A4A5158401808
:10909000A1005050641C102C00DA6FE7FEBD0000E8
:1090A000D00F002090100020900D0020500E0020C6
:1090B000900F00205010002000200FE08100094A8E
:1090C0005158CA01511ACA09011D8900064B595845
:1090D000C90951188200034B9950401C0428EDDB4C
:1090E00070470000C8040020900F002070B50422D3
:1090F00051212748FFF71AF90546A80024494018CE
:1091000044880720000220400412002C03D1402094
:10911000204908802DE0012C03D180201D490880C2
:1091200027E0022C03D1E0011A49088021E0032C3A
:1091300004D101204002174908801AE0042C03D111
:1091400020021449088014E0052C03D1082011499D
:1091500008800EE0062C03D110200E49088008E09C
:10916000072C03D120200B49088002E00AA0FEF75B
:109170004DFE4020074988700120C87005200C4929
:10918000087001200B49087000200B49087070BD61
:10919000380C00209C0400205245475F434F4E543A
:1091A000454E545F6572725F6F70740A0000000074
:1091B000A0040020A1040020A204002070B50446F1
:1091C0000D461646034832462946436820469847CE
:1091D00070BD0000BC03002070B504460D46164665
:1091E00003483246294603682046984770BD000070
:1091F000BC03002010B5002400BF0AE0A000124B01
:10920000C0184288A000195C4020FFF7E5FF601CF1
:1092100084B2A0000C49085A0028EFD10E210B4857
:10922000F8F7A9FF08210A48F8F7A5FF0848FAF758
:10923000BDFC0748408808380449888104494888AB
:10924000FEF78AF910BD0000380C0020100900203C
:10925000600400200020002106E0074A525C012A39
:1092600001D000207047491C044AD27852008A423B
:10927000F3DC012000BFF5E7340C00209C04002043
:1092800010B5FEF715FFFFF731FFFFF77DFA00235A
:109290001A4619461846FFF7B7F900F063F8FFF7CA
:1092A000A9FF10BD7FB505460E466A4631462846E1
:1092B000F9F784F900242CE0002C03D10020184990
:1092C000087002E000201749087003A8005D01281B
:1092D0001ED1002C02D11249087002E00120114970
:1092E000087060006946085E61000F4A515E88425E
:1092F0000EDA60006946085A6100505203A8015D09
:1093000010460C30015509480178104608300155C7
:10931000641C0748C0784000A042CDDC7FBD00003F
:109320009804002099040020280C0020A2040020AA
:109330009C0400200246002013780C2B05DB002340
:1093400013700B785B1C0B7002E013785B1C1370BE
:1093500013780C2B02DC0B78022B01DD012000E0DE
:109360000020704710B56D2251211648FEF7DEFF30
:1093700004461548007880001449085AA100114A93
:1093800089184880702251210E48FEF7CFFF04460D
:109390000D48007880000D4940184088A100094A16
:1093A000891848806E2251210648FEF7BFFF044607
:1093B0000748007840000749085AA100014A891867
:1093C000488010BD380C0020A0040020709A0008CE
:1093D000A1040020A49A000810B50A4800680128DA
:1093E0000FD1FAF7CFFB0848FCF7AAFB0749086042
:1093F0000846016804480068FFF7A2FB0020014905
:10940000086010BD800400207C0400207804002047
:1094100070B504460D467D23DB002A4621460248EE
:10942000FCF7FCFB70BD0000300B00204000074241
:1094300041000400090001E901000000670000008C
:1094400072005006420013004300008844004000B0
:10945000450000004600A00F47000010480010A47F
:10946000490000204A00F82A4B0012004C0058A97D
:109470004D0000004E0001004F0000005000A00F02
:109480005100F400520000245300020A5400D40694
:1094900055000000560024005700FFFF580075FFDC
:1094A000590000005A0000005B0022005C0022000E
:1094B0005D0019195E0000FF6100B5026200B5028F
:1094C0006300B5026400B5026E00FC836600000A0A
:1094D0006C0090996D00C09D7000A03E7600210048
:1094E0000200193004000C00090001610A000002AA
:1094F0000B0019C005001000060049010700B20169
:1095000008001C000D0000100E0000401400035A5B
:1095100015000817170010022000000021000000AD
:10952000220000002300DC1D24005E1D2500E21C3B
:109530002600641C2700D0172800D4162900DC154B
:109540002A00DC152B00DC152C00DC152D00DC15A9
:109550002E00DC152F00DC15720093076700401801
:1095600001002282410044C84000070200000000C0
:10957000AABF1014FDFCFBFAF4F3F2F1F8F7F6F5CC
:109580000000000000000000C409000008070000FF
:10959000080700000807000008070000080700008F
:1095A000080700000807000008070000080700007F
:1095B000080700000807000008070000080700006F
:1095C0004000074241000400090001E901000000D9
:1095D000670000007200500642000100430080381E
:1095E00044004000450000004600A00F4700001066
:1095F000480010A4490000204A00F82A4B0000004F
:109600004C00D8594D0000004E0001004F000000F2
:109610005000A00F5100F400520000245300020A31
:109620005400ABAA55000000560024005700FFFF6D
:10963000580075FF590000005A0000005B0022002E
:109640005C0022005D0019195E0000FF610021002E
:109650006200210063002100640021006E00FC8391
:109660006600000A6C0090996D00C0937000A02AFB
:109670007600210002006E1004000C02090001694E
:109680000A0000420B006EC00500100006004901F0
:109690000700B20108001C000D0000100E00004081
:1096A0001400035A150008171700100220000000CC
:1096B00021000000220000002300DC1D24005E1DAC
:1096C0002500E21C2600641C2700D0172800D416B1
:1096D0002900DC152A00DC152B00DC152C00DC151C
:1096E0002D00DC152E00DC152F00DC157200930711
:1096F000670040180100209E410044C84000070256
:1097000000000000700020106C0080886D00008850
:1097100072005006670000006600F0F06E00FC0367
:1097200041000448000000004000074241000400DE
:10973000090001E901000000670000007200500606
:10974000420003004300802C440008004500000054
:109750004600A00F47000000480028A04900000074
:109760004A0028A04B0001004C0090DC4D00000096
:109770004E0001004F0000005000A00F51006E018C
:10978000520000365300000A54000000550000004B
:10979000560000005700000058000000590000006B
:1097A0005A0000005B0022005C0022005D001919D5
:1097B0005E0000FF6100EF106200EF106300EF1029
:1097C0006400EF106E00B4AB6600000A6C00909964
:1097D0006D0080957000A02E7600210002001920F7
:1097E00004000C01090001650A0000C20B0019C049
:1097F00005001000060049010700B20108001C0026
:109800000D0000800E0000081400035A1500081710
:1098100017001002200000002100000022000000BC
:109820002300DC1D24005E1D2500E21C2600641CB4
:109830002700D0172800D4162900DC152A00DC15D3
:109840002B00DC152C00DC152D00DC152E00DC15A2
:109850002F00DC1572009307670040180100248E6A
:10986000410044C8400007020000000040008000A2
:10987000000100020004700020106C0080886D0060
:10988000008872005006670000006600F0F06E006D
:10989000FC03410064C800000000410044C872009D
:1098A00053066C0090996D00C0937000A02A6E0062
:1098B000FC836600000A670040186900060000008B
:1098C00000000000E1620008C75D00080000000021
:1098D0000000000000000000000000000000000088
:1098E0000000000000000000000000000100000077
:1098F0000200000003000000040000000600000059
:10990000070000000800000009000000000000003F
:109910000000000000000000000000000100000046
:1099200002000000030000000400000040000742A5
:1099300041000400090001E9010000006700000087
:1099400072005006420013004300008844004000AB
:10995000450000004600A00F47000010480010A47A
:10996000490000204A00F82A4B0012004C0058A978
:109970004D0000004E0001004F0000005000A00FFD
:109980005100F400520000245300020A5400D4068F
:1099900055000000560024005700FFFF580075FFD7
:1099A000590000005A0000005B0022005C00220009
:1099B0005D0019195E0000FF6100B5026200B5028A
:1099C0006300B5026400B5026E00FC836600000A05
:1099D0006C0090996D00C09D7000A03E7600210043
:1099E0000200193004000C00090001610A000002A5
:1099F0000B0019C005001000060049010700B20164
:109A000008001C000D0000100E0000401400035A56
:109A100015000817170010022000000021000000A8
:109A2000220000002300DC1D24005E1D2500E21C36
:109A30002600641C2700D0172800D4162900DC1546
:109A40002A00DC152B00DC152C00DC152D00DC15A4
:109A50002E00DC152F00DC157200930767004018FC
:109A600001002282410044C84000070200000000BB
:109A7000C09DA03EC09FA036C099A032C097A02E26
:109A8000C097A02AC093A02AC097A026C09FA0225A
:109A9000C09BA022C099A022C097A0228097A02E90
:109AA0008095A02EFC839083B4AB000060C20500BB
:109AB00090F3020000410000B8250000B825000026
:109AC000B8250000B8250000B8250000B825000022
:109AD000B8250000B8250000B8250000B825000012
:109AE000B8250000B8250000B825000000040000DB
:109AF000EC030000B203000053030000D402000096
:109B00003902000088010000C800000000000000C9
:109B100038FFFFFF78FEFFFFC7FDFFFF2CFDFFFFB3
:109B2000ADFCFFFF4EFCFFFF14FCFFFF0000000038
:109B3000C80000008801000039020000D4020000C3
:109B400053030000B2030000EC0300000004000017
:109B5000EC030000B203000053030000D402000035
:109B60003902000088010000C80000008C9B00083A
:109B7000000000201C05000048240008AC9D0008DF
:109B80001C050020D4100000D07E000801C71A0177
:109B90000171130801690B91126D144095701BA09F
:109BA0002A084A97082A80101A22105A9B1829104E
:109BB0001A2E181A91081A26089A992019185B402B
:109BC0009D204A9F18394029282950693029085A70
:109BD0009360293829102930692829182928698093
:109BE0002950291819082AC00819581BC0F5081A45
:109BF0002708294029105970392019485AC060395E
:109C0000106908294029585A32301A360829B013E9
:109C10003E611CEF1062041A63041A6404126E1B86
:109C2000B4AB141A03141A03141A031413036E1496
:109C300090836112211A62041A63041A6404126E7A
:109C40001AFC141CB50262041A63041A6404291471
:109C500021A009FDFCFBFA0403020192641A320CF4
:109C6000129612C812FA303C2C015E019001C2011A
:109C7000F401260258028A02BC02EE0220035203BB
:109C80008403B603E803FC031004240438044C04E2
:109C90006004740488049C04B004BC076009B40A1E
:109CA000860BFF13FD30420832FE4B1D310C32EFA4
:109CB0004BD5240C32EE5AA10C415A313032125A93
:109CC0003D3029A14B91320C32024B992F0C32FDC1
:109CD0005A69302A0730592429055A4D2432095A25
:109CE0007D24320A4B9D2C0C32605AAD6032614BA0
:109CF000A92E0C32645AF7482A107C4A330C3211D0
:109D00005A054832144B6D2B0C727513413773088A
:109D10007113F9367308701AC50C72741A75242AF7
:109D20002748599C0312FFFF157956341235550107
:109D30000A0514ED230123999523DE0C1A77E10916
:109D40002E04147F9501230BA5232F342390120B8F
:109D50002C480904013553127A3204F2011305012B
:109D60001A080111A23C03130752CB7602041252C7
:109D7000125C127812A612E4181630018501E20175
:109D800041029F02F80249038E03C503EA03FE0263
:109D90001AEA0A1E8E034903F81A1C4102E2261C25
:0C9DA0003001E4321A783A4962000000F9
:209DC000FFFFFFFFFFFFFFFFFFFFFFFFFFFFFFFFFFFFFFFFFFFFFFFFFFFFFFFFFFFFFFFFA3
:209DE000FFFFFFFFFFFFFFFFFFFFFFFFFFFFFFFFFFFFFFFFFFFFFFFFFFFFFFFFFFFFFFFF83
:209E0000FFFFFFFFFFFFFFFFFFFFFFFFFFFFFFFFFFFFFFFFFFFFFFFFFFFFFFFFFFFFFFFF62
:209E2000FFFFFFFFFFFFFFFFFFFFFFFFFFFFFFFFFFFFFFFFFFFFFFFFFFFFFFFFFFFFFFFF42
:20AC0000795634120055010A05000000ED23010099950000DE0C0000770700007707000095
:20AC2000770700007707000077070000770700007707000077070000770700007707000024
:20AC40007707000077070000770700007F9501000BA500002F34000090120000480900005F
:20AC600048090000480900004809000048090000480900004809000048090000480900004C
:20AC80004809000048090000480900000000000000000000000000000000000000000000C1
:20ACA000000000000000000000000000000000000000000000000000000000000000000094
:20ACC00000366E010E000000030000000100000000000000000000000000000005010008AF
:20ACE000080808003C000000000000000000000752000000000000000000000000000000A7
:20AD0000FFFFFFFFFFFFFFFFFFFFFFFFFFFFFFFFFFFFFFFFFFFFFFFFFFFFFFFFFFFFFFFF53
:20AD2000FFFFFFFFFFFFFFFFFFFFFFFFFFFFFFFFFFFFFFFFFFFFFFFFFFFFFFFFFFFFFFFF33
:20AD4000FFFFFFFFFFFFFFFFFFFFFFFFFFFFFFFFFFFFFFFFFFFFFFFFFFFFFFFFFFFFFFFF13
:20AD6000FFFFFFFFFFFFFFFFFFFFFFFFFFFFFFFFFFFFFFFFFFFFFFFFFFFFFFFFFFFFFFFFF3
:20AD8000FFFFFFFFFFFFFFFFFFFFFFFFFFFFFFFFFFFFFFFFFFFFFFFFFFFFFFFFFFFFFFFFD3
:20ADA000FFFFFFFFFFFFFFFFFFFFFFFFFFFFFFFFFFFFFFFFFFFFFFFFFFFFFFFFFFFFFFFFB3
:20ADC000FFFFFFFFFFFFFFFFFFFFFFFFFFFFFFFFFFFFFFFFFFFFFFFFFFFFFFFFFFFFFFFF93
:20ADE000FFFFFFFFFFFFFFFFFFFFFFFFFFFFFFFFFFFFFFFFFFFFFFFFFFFFFFFFFFFFFFFF73
:20AE0000FFFFFFFFFFFFFFFFFFFFFFFFFFFFFFFFFFFFFFFFFFFFFFFFFFFFFFFFFFFFFFFF52
:20AE2000FFFFFFFFFFFFFFFFFFFFFFFFFFFFFFFFFFFFFFFFFFFFFFFFFFFFFFFFFFFFFFFF32
:20AE4000FFFFFFFFFFFFFFFFFFFFFFFFFFFFFFFFFFFFFFFFFFFFFFFFFFFFFFFFFFFFFFFF12
:20AE6000FFFFFFFFFFFFFFFFFFFFFFFFFFFFFFFFFFFFFFFFFFFFFFFFFFFFFFFFFFFFFFFFF2
:20AE8000FFFFFFFFFFFFFFFFFFFFFFFFFFFFFFFFFFFFFFFFFFFFFFFFFFFFFFFFFFFFFFFFD2
:20AEA000FFFFFFFFFFFFFFFFFFFFFFFFFFFFFFFFFFFFFFFFFFFFFFFFFFFFFFFFFFFFFFFFB2
:20AEC000FFFFFFFFFFFFFFFFFFFFFFFFFFFFFFFFFFFFFFFFFFFFFFFFFFFFFFFFFFFFFFFF92
:20AEE000FFFFFFFFFFFFFFFFFFFFFFFFFFFFFFFFFFFFFFFFFFFFFFFFFFFFFFFFFFFFFFFF72
:20AF000001000000FFFFFFFFFFFFFFFFFFFFFFFFFFFFFFFFFFFFFFFFFFFFFFFFFFFFFFFF4C
:20AF2000FFFFFFFFFFFFFFFFFFFFFFFFFFFFFFFFFFFFFFFFFFFFFFFFFFFFFFFFFFFFFFFF31
:20AF4000FFFFFFFFFFFFFFFFFFFFFFFFFFFFFFFFFFFFFFFFFFFFFFFFFFFFFFFFFFFFFFFF11
:20AF6000FFFFFFFFFFFFFFFFFFFFFFFFFFFFFFFFFFFFFFFFFFFFFFFFFFFFFFFFFFFFFFFFF1
:20AF8000FFFFFFFFFFFFFFFFFFFFFFFFFFFFFFFFFFFFFFFFFFFFFFFFFFFFFFFFFFFFFFFFD1
:00000001FF
